:100000000C946F000C9400000C9400000C94000001
:100010000C9400000C9400000C9400000C94000060
:100020000C9400000C9400000C9400000C94000050
:100030000C9400000C9400000C9400000C94000040
:100040000C94D1000C9400000C949E000C940000C1
:100050000C9400000C9400000C9400000C94000020
:100060000C9400000C9400001027E80364000A00C0
:1000700001000010000110000100000000000A0053
:100080000000000000000000000000000000000070
:100090000000000000000000000000000000000060
:1000A0000000000000000000000000000000000050
:1000B000000000000000000000000A0A0A0A0A0A04
:1000C0000A0A0A0A0A0A0A0A0A0A020002007A004E
:1000D000020004007C00010007037E000000F89489
:1000E000EE27EFBBF1E0F5BFE5BF8DE0A2E0BB2757
:1000F000ED938A95E9F780E098E0A0E0B1E0ED9318
:100100000197E9F7EAECF0E085919591009761F0AD
:10011000A591B59105901590BF01F00105900D9244
:100120000197E1F7FB01F0CFE8E0EEBBEFEFEDBFA9
:10013000E8E0EEBFC0E0D3E00C94BA03AA93EA93E0
:10014000FA93EFB7EA931A930A931091C0000091C3
:10015000C600E12FEC71E9F4E091F903EF5FE09361
:10016000F903E150F0E0E052FC4F0083A091F90365
:10017000A93119F4E0E0E093F903A091FB03AF5F2C
:10018000A093FB03A93129F4E0E0E093FB0368941A
:1001900037F809911991E991EFBFF991E991A99186
:1001A00018950A921A926A937A938A939A93AA93C9
:1001B000BA93EA93FA93EFB7EA93E0913E03F09192
:1001C0003F033196E0933E03F0933F030E941326D2
:1001D000E1E5F1E00E94D4310E2E0E941326E3EAFD
:1001E000F2E00E94D431E02909F40BC2A0913C0353
:1001F000B0913D03E5E0F0E00E94F2310E2EA091B7
:100200002203EEE00E94CA31E02121F0E0912203B6
:10021000EF5F03C025FC03C0E0E0E0932203A09160
:100220002203AE3011F4689425F8A0912B03A1307D
:1002300029F4F79B02C0F79801C0F79AE1E02E2657
:100240000E9418260E942126E093C403F093C50360
:100250006093C6037093C7030E942826A8EAB3E000
:100260000E942D260E943426A4EDB3E00E942D2684
:100270000E9439260E9442260E94FB30E093A80388
:10028000F093A9036093AA037093AB03A091D403E6
:10029000B091D5038091D6039091D703E0E0F0E0D0
:1002A00060E772E40E94FB30E093D403F093D5033F
:1002B0006093D6037093D7030E9447260E944C2672
:1002C0000E2E0E9451260E944C26E02161F1E09101
:1002D000D403F091D5036091D6037091D7030E94A7
:1002E00039260E94FB30E093D003F093D103609352
:1002F000D2037093D3030E945626A0E5B3E00E9478
:100300005F26A091D003B091D1038091D203909148
:10031000D3030E942126E093B003F093B1036093CE
:10032000B2037093B3030E9464260E9475260E9454
:100330005D30E093B803F093B9036093BA03709310
:10034000BB030E9464260E947E260E945D30E093DB
:10035000DC03F093DD036093DE037093DF030E9400
:1003600087260E9490260E94A326A0E9B3E00E945F
:10037000EC2F0E94DC320E948726AAE0B0E080E0E9
:1003800090E00E9420320E947E260E9421300E942E
:10039000403170F0E0E0E093DC03E093DD03E093B4
:1003A000DE03E093DF030E94A82631960E94AD266B
:1003B000E0919403F09195036091960370919703F7
:1003C000A091BC03B091BD038091BE039091BF0387
:1003D0000E94AD30DF01CB010E942126E093C803CB
:1003E000F093C9036093CA037093CB030E94B226B3
:1003F0000E945D300E94BB26E0910E03F0E00E9457
:10040000C4260E94A2310E94CD26A0E7B3E00E943C
:10041000DC260E9418260E943C333CF5A091C803BC
:10042000B091C9038091CA039091CB030E94E12649
:100430007F936F93FF93EF93A091C403B091C50393
:100440008091C6039091C7030E94E126AF91BF91AE
:100450008F919F910E94FB30E093C003F093C10302
:100460006093C2037093C30309C0E0E0E093C0034C
:10047000E093C103E093C203E093C303A091C303DD
:10048000AA238AF40E94E8260E94F12618F40E940A
:10049000F82608C00E94FF260E94B72FA8E7B3E005
:1004A0000E94DC2614C00E94E826E0E0F0EC69E738
:1004B00074E40E94403109F008F403C00E94F82659
:1004C00006C00E94FF26A8E7B3E00E94DC260E9437
:1004D00008270E9411270E945D300E941A27E09190
:1004E000A803F091A9036091AA037091AB030E9445
:1004F00023270E94403168F5E091B003F091B103E9
:100500006091B2037091B3030E9423270E945D3073
:10051000E093AC03F093AD036093AE037093AF032D
:100520000E9423270E942C270E945630DF01CB0116
:100530000E9456260E94FB30A0E0B0E081E695E4E0
:100540000E94AD30ACE6B3E00E94DC26689424F84B
:1005500002C0E0E12E260E9408270E9435270E9453
:100560005D30E093B403F093B5036093B6037093EA
:10057000B7030E943527E0E0F0E060E87FE30E94E7
:10058000403109F008F412C0E093B403E093B503DE
:10059000E093B603E093B7030E943E27EF5FFF4F5F
:1005A0006F4F7F4F0E9447270E9450270E94562777
:1005B000A034E2E4BE07EFE08E07E0E09E0778F0AB
:1005C000E0E0E0935E03E0935F03E0936003E09379
:1005D0006103A2E4B0E00E945F270E9411330E94F1
:1005E00011270E946427A0E4B3E00E945F26A09137
:1005F0002003AC3308F4F298A0912003AC3309F443
:10060000F29A0E941326A33AE2E0BE0709F089C0DD
:10061000A0911F030E9468270E946D270E945F27F8
:100620000E94F8310E947627E02191F0E0912003AA
:10063000EF5FE0932003E0911F03F0E03296A0917A
:100640002003B0E0EA17FB0719F4ECE3E093200382
:10065000E0E0E0933E03E0933F03D394A0910F03C7
:10066000A13028F4E0910F03EF5FE0930F030E94A5
:100670007D27E8E5F2E00E94EC310E2E0E948227F1
:10068000E021E9F0E0915403F09155033196E093B5
:100690005403F09355030E947D270E948727EA1B8D
:1006A000FB0BE0935A03F0935B030E946D270E94BB
:1006B0003C332CF4E0E0E0935403E0935503ECE387
:1006C000ED1589F4DD24C394EC1569F4CC24E09194
:1006D0000003EF5FE0930003A0910003A43119F43D
:1006E000E0E0E0930003A0912703A130D0F0E09177
:1006F0001203EF5FE0931203A0911203A23088F07F
:10070000E0911103EF5FE0931103E0E0E093120347
:10071000E0912703A0911103EA1718F4E0E0E093B9
:100720001103E991EFBFF991E991B991A9919991DB
:10073000899179916991199009901895AA93E88106
:10074000E066E0937C0085E28A95F1F7E0917A001B
:10075000E064E0937A00E0917A00E071E1F3E091E7
:100760007A00E061E0937A00E0917800F0917900FE
:1007700021960895EF9761978AE4A6E0B0E0E0E85B
:10078000F0E00E945133FF2401E021E0E0E8E09333
:100790006100E0E0E0936100EFE0E4B9E1E0E5B999
:1007A000E0E0E7B9E4E0E8B9EAEFEAB9E7EEEBB98F
:1007B000E0E0E4BDE3E0E5BDE0E0E6BDE7BDE8BDC7
:1007C000E0938000E0938100E0938500E093840053
:1007D000E0938700E0938600E0938900E09388002F
:1007E000E0938B00E0938A00E093B600E1EAE093A7
:1007F000B000E2E0E093B100E0E0E093B200E0930B
:10080000B300E093B400E1E0E0936E00E0E0E09339
:100810006F00E0937000E0936900EDBBE093680027
:10082000E093C000E8E9E093C100E6E0E093C20095
:10083000E0E0E093C500E7E4E093C400E0E8E0BF57
:10084000E0E0E0937F00E0937E00E0E6E0937C0050
:10085000E6E2E0937A00E0E0E0937B00ECBDE09319
:10086000BC0078945F9A0E948C270E9490270E9477
:1008700096270E949D270E94AA270E948C27EAE0C3
:100880006E1668F4AEE2B0E00E94B727A8E2B0E0CE
:10089000E0E00E942133A9E2B0E00E942133EAE0C7
:1008A0009E1650F4A4E3B0E00E94B727ACE3B0E09A
:1008B0000E94B727689426F8EAE0BE1618F46894F8
:1008C00030F827F8689433F8E7E1E09314030E94C6
:1008D000BC270E94C3270E94CA27E8ECF0E0E093FF
:1008E0006603F0936703A0E0B0E00E940533E09355
:1008F0001503A1E0B0E00E940533E0931603A2E0E7
:10090000B0E00E940533E0931703A3E0B0E00E943B
:100910000533E0931903A4E0B0E00E940533EEA391
:10092000A5E0B0E00E940533EFA3A6E0B0E00E948E
:100930000533E8A7A7E0B0E00E940533E0931A036F
:10094000A8E0B0E00E940533E0931B03A9E0B0E00B
:100950000E940533E0931C03F798F198AAE0B0E0F9
:100960000E940533E0931F03ACE2B0E00E94013324
:100970000E94D127A4E1B0E00E940533EAA3A5E1DB
:10098000B0E00E940533EBA3A6E1B0E00E9405337E
:10099000ECA3ABE0B0E00E940533EE8FACE0B0E03A
:1009A0000E940533EF8FADE0B0E00E940533E8A36D
:1009B000A0E3B0E00E940133EF87F88BAEE0B0E037
:1009C0000E940533E0932C03AFE0B0E00E940533B2
:1009D000E0932E03A0E1B0E00E940533E0932D03E5
:1009E000A2E4B0E00E94FD320E944727AEE2B0E0F0
:1009F0000E940133A4EAB3E00E94D6270E942C276C
:100A0000A0E4B3E00E945F260E9411270E944226C4
:100A10000E94FB300E941A27A1E1B0E00E9405333A
:100A20003E2FA2E3B0E00E940133EB8BFC8BA2E1EE
:100A3000B0E00E940533EAA7A3E1B0E00E940533CD
:100A4000E9A7A4E3B0E00E940133A8EBB3E00E9461
:100A5000D627ACE3B0E00E940133A8EDB3E00E94DA
:100A6000D6270E94B2260E9442260E94FB300E9496
:100A7000BB26A6E3B0E00E9401330E94DD27AAE373
:100A8000B0E00E9401330E94A2310E94E227A7E158
:100A9000B0E00E9405330E944C3323F8A8E3B0E095
:100AA0000E9401330E94EB27A8E1B0E00E940533C9
:100AB000E0930603A9E1B0E00E940533E093080348
:100AC000AAE1B0E00E940533E0930903ABE1B0E096
:100AD0000E940533E0930A03ACE1B0E00E940533C5
:100AE000E0930B03ADE1B0E00E940533E0930C030B
:100AF000AEE1B0E00E940533E0932303AFE1B0E044
:100B00000E940533E0932403A0E2B0E00E94053385
:100B1000E0932503A1E2B0E00E940533E0932603B1
:100B2000A2E2B0E00E940533E0932703A3E2B0E025
:100B30000E940533E0932803A4E2B0E00E9405334D
:100B4000E0932903A5E2B0E00E940533E0932A0375
:100B5000AEE3B0E00E9401330E94AD26A6E2B0E011
:100B60000E940533E0930E03A7E2B0E00E94053334
:100B70000E944C3336F8AAE2B0E00E940533E093BD
:100B80001003ABE2B0E00E940533E98FA0E4B0E0CF
:100B90000E940133EB87FC8736FE0BC0A8E2B0E071
:100BA0000E940533CE2EA9E2B0E00E940533E09307
:100BB0000003A0910203AE3128F4E0910203EF5F3D
:100BC000E0930203A0910203AE31A1F4E0E0E093D0
:100BD0003103E0933203EBE0F0E0E0935803F0934D
:100BE0005903E8EBE0933303E0E0E093F903E4E139
:100BF000E0930203A091F903AB30E1F4E091E2034A
:100C0000E0933003E091E303E0933103E091E403E8
:100C1000E0933203E091E503F0E0E0935803F093B2
:100C20005903E091E603E0933303E0E0E093F90336
:100C3000E0930203A091F903AC30C0F0E0E0E09350
:100C4000E003E093E103E093E203E093E303E09346
:100C5000E4030E94BC27E0E0E093E703E093E803AD
:100C6000E093E903E093EA03E093F903E8EC5E160E
:100C700030F45394E4E1E51511F4E1E04E2E0E94C6
:100C8000F027E7EAE0937A00A6E00E94F427EF83DA
:100C9000F887E7E2E0937A000E94F0270E9490270D
:100CA0000E9497310E949331E987FA87E7E2E09347
:100CB0007A000E94F0270E94FB273B97A0F1A0E05A
:100CC0000E94F427662777270E940428A8EEB3E045
:100CD00080E090E00E944B32DF01CB010E940D28A2
:100CE000662777270E948D320E940428A4E9B3E08A
:100CF0000E9423300E94DC32E0910703EF5FE09313
:100D00000703E0910603A0910703AE1750F00E947D
:100D10001228E0938C03F0938D0360938E037093FD
:100D20008F03E894F3F80E941B280E9490270E94EA
:100D300096270E942228A2E00E94F427DF01E5E026
:100D4000F0E00E9450328E2E0E941B280E94AA279B
:100D50008AE48A95F1F70E949D270E9422280E942A
:100D600029280E941B28E7EAE0937A00A5E0E6DC48
:100D7000EF2FF0E01E2F0E941B280E94FB27AE2EB3
:100D80000E941B28E0911003E03009F091C0E1E0DF
:100D9000E51589F50E9433285E9710F4E1E0EC8FA9
:100DA0000E943328E2E3F0E00E94F2310E2E0E940E
:100DB0003328EAEFF0E00E94EC31E02111F0E2E0AC
:100DC000EC8F0E943328AB3FE0E0BE0710F0E3E079
:100DD000EC8F1E3110F4E1E0EB8F0E943828A12F38
:100DE000EAEF0E94CA31E02111F0E2E0EB8F1B3FF5
:100DF00010F0E3E0EB8F0E943328EEE1F0E00E9478
:100E0000EC310E943E2811F0E4E00AC00E94332831
:100E1000EAEFF0E00E94F2310E943E2811F0E5E096
:100E2000EC8FA12FEEE10E94CA310E944A2811F0F6
:100E3000E4E008C0A12FEAEF0E94CF310E944A28C7
:100E400011F0E5E0EB8FAC8D0E946827AC8D0E941D
:100E5000562849F0E12F0E945B2818E2AE81AC359C
:100E600011F40E946128AC8D0E946728AC8DE5E0EA
:100E70000E94AC31E02911F00E946128AB8D0E94E4
:100E80006827AB8D0E94562851F018E2AC8D0E9465
:100E90006827AC8D0E94562811F00E946128AB8D06
:100EA0000E9467280E946C28E02909F01CE303C017
:100EB000E0E0EC8FEB8F0E9471280E9477280E945F
:100EC000CA31E021E1F0E4E1EF8B6894F3F80130FE
:100ED00021F4F398F49A02E012C0023059F4F49825
:100EE000F59AA8A5A13010F003E003C0F598F39A95
:100EF00001E005C0033019F4F598F39A01E00E946F
:100F00003328D39708F453C00E9481280E94862872
:100F1000E02F0E948D2810F00E94A028E02F0E9450
:100F2000A7280E94BB28AC91A13008F43FC00E94C2
:100F3000C2280E94CB280E9447334CF40E94BB2851
:100F40000E94D7280E946C310E94E12823C00E9491
:100F5000EA280E94EC28EF930E94EA280E94F528D4
:100F6000AF91EA2379F00E94BB280E94D7280E9403
:100F70007131A0937C03B0937D0380937E039093A3
:100F80007F0308C00E94EA280E94FE281CF00E94ED
:100F900008290CC0A0917C03B0917D0380917E0351
:100FA00090917F030E9417290E941C2904C00E946F
:100FB00061280E9408290E9423290E9429290E22C3
:100FC0000E942E2901F10E9433280E94383310F428
:100FD000E4E1ED8BA09121030E9468270E9436294D
:100FE000E02141F0E3E0E0932F03E0E0E093210310
:100FF0000E943C29E0913803E09321036894F0F8C3
:1010000021F8E894F4F8A0912903A13069F50E9431
:1010100042290E2EA0912103E8EC0E94CA310E94C1
:10102000442939F0F4FE05C0E0912103EF5FE0931D
:101030002103A12FE3E30E94CF310E2EE0E50E94B1
:10104000CA310E22A0912103E0E00E94CF310E941C
:10105000442951F0E0912103E150E093210325FE62
:1010600003C0E3E00E944D290E9436290E2EA12FD5
:101070000E945029A09121030E94552921F0E0E00F
:10108000E093220306C0A0912203A23010F4E8945A
:1010900025F8A0912103A13020F0E0912103F0E098
:1010A00002C00E948128E0933C03F0933D030E941C
:1010B0008128309729F4E89421F86894F4F816C050
:1010C000A0E021FCA1E00E945A290E9442290E22A0
:1010D000A09129030E94552949F0E0E0E093210303
:1010E0000E946128E89422F8689421F8E0910403B2
:1010F0000E943328F0E0EA17FB0720F4E091380360
:10110000E09304030E945F290E9410320E22A091F6
:101110002C030E9455291E2E0E945F290E9408322E
:101120000E22A0912D030E945529E12979F0E0912A
:101130003803E0930403A0E025FCA1E00E946E299F
:101140000E94732919F0E2E00E944D29A091210329
:10115000A13078F0689422F80E948128A0912103A0
:10116000B0E0AE17BF0720F0E09121030E945B289A
:1011700002C0E89422F80E9477290E22A0E031FCF8
:10118000A1E00E94552931F0689431F80E9481282D
:101190000E948D290E947729E02161F10E94922905
:1011A0000E949A29A4F0A0918803B0918903EF8549
:1011B000F889EA1BFB0BA3E0B0E00E9446320E94D4
:1011C000A229AE1BBF0BA0936803B09369030E94D2
:1011D00092290E943C332CF40E94A72932970E9446
:1011E0008D29A0916903AA232AF4E0E0E093680323
:1011F000E09369030E94AC290E94423374F50E9477
:10120000AC290E9471310E949A2974F0AF85B88987
:10121000E0918803F0918903EA1BFB0B0E94A2294D
:10122000EA0FFB1F0E948D290E94AC290E94713198
:10123000A230E0E0BE07E0E08E07E0E09E072CF081
:101240000E94A72931960E948D290E94A229A93CBB
:10125000E0E0BE0714F00E94C3270E94A7290E9465
:101260003328AE17BF0710F4E89431F80E94A7297D
:101270000E943328EA17FB0720F40E94A7290E9446
:10128000B9290E94BE290E9466310E2EA0E032FCD0
:10129000A1E00E94552941F0689432F80E94CD29BE
:1012A000E0936A03F0936B030E94BE290E944031D1
:1012B00009F008F435C00E94D229DF01CB01E0E03B
:1012C000F0E060E070E40E94403109F008F410C0E2
:1012D0000E94D229A0E0B0E080E890E40E94AD3006
:1012E0000E94E1290E94E629AAE6B3E00E94DC26DA
:1012F0000E94D2290E94323354F4EAA5F0E00E9401
:10130000E129AE1BBF0BA0936A03B0936B03A091BE
:101310006B03AA232AF4E0E0E0936A03E0936B03F3
:101320000E94BE290E944031C0F50E94EB29DF01D6
:10133000CB01E0E0F0E060E470E40E94403109F0AD
:1013400008F414C00E94EB29A0E0B0E080EA90E429
:101350000E94AD30DF01CB010E94F6290E94FB29DB
:101360000E945D30AAE6B3E00E94DC260E94EB29D1
:101370000E94323354F4E9A5F0E00E94E129EA0F1B
:10138000FB1FE0936A03F0936B030E94E129A13DE8
:10139000E7E0BE0714F00E94CA270E94CD29DF01B2
:1013A0000E94F629AE17BF0710F4E89432F80E94A5
:1013B000CD29DF010E94F629EA17FB0720F40E94DD
:1013C000E1290E94002A0E94052A0E9410320E2E56
:1013D000A0E034FCA1E00E94552931F0689434F873
:1013E0000E94CD290E940C2A0E94052A0E944233A5
:1013F0005CF50E94112A0E949A299CF0E091160344
:10140000F0E0A0918403B0918503AE1BBF0BE3E035
:10141000F0E00E941A2AAE1BBF0BA0937203B09398
:1014200073030E94112A0E943C332CF40E94212A4B
:1014300032970E940C2AA0917303AA232AF4E0E0B9
:10144000E0937203E09373030E94052A0E944733DE
:101450008CF50E94262AA430E0E0BE07E0E08E076B
:10146000E0E09E078CF0A0911603BB27E091840377
:10147000F0918503AE1BBF0BE2E0F0E00E941A2A58
:10148000EA0FFB1F0E940C2A0E94262A0E943C336E
:101490002CF40E94212A32960E940C2AA0917203F9
:1014A000B0917303A13DE7E0BE0724F0E0EDF7E063
:1014B0000E940C2A0E94CD29DF010E94212AAE172A
:1014C000BF0710F4E89434F80E94CD29DF010E9490
:1014D000212AEA17FB0730F4A0917203B09173033D
:1014E0000E94002AE09113030E943328F0E0EA17DB
:1014F000FB0720F4E0913803E0931303E09113031A
:10150000F0E035970E9433280E94EC316E2F0E2EAA
:10151000A0E031FCA1E00E94362A1E2E062EA0E09B
:1015200032FCA1E00E94362A1E2A062EA0E034FCDE
:10153000A1E00E94362AE12949F0E0913803E093C6
:10154000130325FE03C0E2E00E944D29A0912F0362
:10155000A13078F00E946128A0912F03A13021F4DE
:10156000EAE0F0E00E94B929E0912F03E150E09316
:101570002F030E943828A09129030E9455291E2E6E
:10158000A12FE0E50E94CF310E2EA0912903E1E0CA
:101590000E94AC310E9444291E2A0E943828A09142
:1015A0002903E1E00E94AC310E220E947329E12957
:1015B000E1F0E0E0E0930503A0912103A13018F0F1
:1015C000E2E0E0932F03E0E0E0932103E12FF0E07D
:1015D000F2970E94FB29A6EFB8E28CE99FE30E94F4
:1015E000AD300E94EA2F1E2F01C010E00E9481281A
:1015F000ED87FE87A12F0E946827A09124030E94F7
:10160000362A11F0299A01C02998A82DE4E60E94F3
:10161000CA316E2F0E2E0E943B2A0E22AE81EDE5BE
:101620000E94B1310E94422A1E2E062E0E943B2AA1
:101630000E220E942929E0211E2A0E9487270E944B
:101640007D270E94D4310E94492A0E948227E021EE
:10165000E12931F1E0914003F0914103AEE2B0E0C5
:101660000E94512A0E94572A0E94B2260E94642793
:101670000E94642A0E94692AEC2DA8E2B0E00E9430
:101680006D2AE0910003A9E2B0E00E9421330E949C
:101690008C275F98A8EEB3E00E94AD2F5F98FECF35
:1016A000AB2D0E94732A0E942929E02131F0E89491
:1016B000F2F827F8E0E0E09337030E94782A0E94CE
:1016C0002929E02171F0E0913703EF5FE0933703C0
:1016D000A0913703AA3029F4E0E0E0933703E093C8
:1016E0002B030E94782AA0E0F2FCA1E00E9450297E
:1016F0000E942929E02191F1E4E1EE8B6894F2F84F
:10170000E0912B03EF5FE0932B030E94812A0E945C
:101710002E2919F0E1E0E0932B03A0912B030E9406
:1017200067280E942E2919F0E2E0E0932B030E9423
:10173000812AA09124030E94552919F0E1E0E09349
:101740002B03A0912B030E946728A0E0F0FCA1E0EE
:101750000E94362A19F0E3E0E0932B03E0912B037B
:10176000E03031F4E0E0E093B400F7982A981DC02F
:10177000A0912B03A13031F4E0911C03E093B4005D
:101780002A9813C0A0912B03A23031F4F79AEFEFFF
:10179000E093B4002A9809C0A0912B03A33029F448
:1017A000F79AEFEFE093B4002A9A0E9442290E2E96
:1017B000A12FE0E00E94CF310E220E94732929F16F
:1017C000A0912303A13009F45C9AE0910303EF5F39
:1017D000E0930303A0910303E5E00E94CF310E2EB6
:1017E000E4E10E94CA31E02141F0E0910303E1709D
:1017F000AFEFEA02F001E093B400A0910303A0313F
:1018000018F0E0E0E093030325C05C98A0E030FC12
:10181000A1E00E946E29A0912B030E945529D1F0CE
:10182000E0913603EF5FE0933603A0913603A130D9
:1018300019F4EFEFE093B400A0913603A33019F44C
:10184000E0E0E093B400A0913603A43019F4E0E0A6
:10185000E0933603E0911B03E093B300EAE0E9155F
:1018600018F4E894F1F826F80E94882AA0E026FCF3
:10187000A1E00E945029A0E0F1FCA1E00E945029C3
:101880000E942929E02139F16894F1F8E0910D03D3
:10189000EF5FE0930D03E0E0EA8FAA8DA53088F4B6
:1018A0000E948E2AA081A13018F0E5E0EA8F05C0E1
:1018B000E0910D03EF5FE0930D03EA8DEF5FEA8F98
:1018C000ECCFA0910D03A53018F0E0E0E0930D03FC
:1018D0000E948E2A20810E94882AA0911E03EFEF89
:1018E0000E94CA31E02121F0E0911E03EF5F03C0A6
:1018F000E894F1F8E0E0E0931E03A0911E03A43108
:1019000009F03FC1AE81E0E00E94C0310E2E0E947E
:101910002929E02119F0EE81E150EE83233610F4FD
:1019200023E62FC121E0E0E0E0930D03E0911503F1
:10193000A0E0B0E00E946D2AE0911603A1E0B0E0C3
:101940000E946D2AE0911703A2E0B0E00E946D2A88
:10195000E0911903A3E0B0E00E946D2AEEA1A4E09B
:10196000B0E00E946D2AEFA1A5E0B0E00E946D2AD0
:10197000E8A5A6E0B0E00E946D2AE0911A03A7E076
:10198000B0E00E946D2AE0911B03A8E0B0E00E9445
:101990006D2AE0911C03A9E0B0E00E946D2AE0915D
:1019A0001F03AAE0B0E00E946D2A0E940D28ACE25D
:1019B000B0E00E94512AEAA1A4E1B0E00E946D2AA1
:1019C000EBA1A5E1B0E00E946D2AECA1A6E1B0E098
:1019D0000E946D2AEE8DABE0B0E00E946D2AEF8D83
:1019E000ACE0B0E00E946D2AE8A1ADE0B0E00E945A
:1019F0006D2AEF85F889A0E3B0E00E94512AE091BA
:101A00002C03AEE0B0E00E946D2AE0912E03AFE01F
:101A1000B0E00E946D2AE0912D03A0E1B0E00E94A9
:101A20006D2AE32FA1E1B0E00E946D2AEB89FC89C9
:101A3000A2E3B0E00E94512AEAA5A2E1B0E00E9430
:101A40006D2AE9A5A3E1B0E00E946D2A0E94572A01
:101A50000E94942AA6E3B0E00E94512AE09162031A
:101A6000F0916303AAE3B0E00E94512AE0E023FC76
:101A7000E1E0A7E1B0E00E946D2A0E948727A8E379
:101A8000B0E00E94512AE0910603A8E1B0E00E9474
:101A90006D2AE0910803A9E1B0E00E946D2AE0916F
:101AA0000903AAE1B0E00E946D2AE0910A03ABE1CC
:101AB000B0E00E946D2AE0910B03ACE1B0E00E941F
:101AC0006D2AE0910C03ADE1B0E00E946D2A0E9406
:101AD000B2260E9464270E94642AE0912303AEE1AB
:101AE000B0E00E946D2AE0912403AFE1B0E00E94D3
:101AF0006D2AE0912503A0E2B0E00E946D2AE091FA
:101B00002603A1E2B0E00E946D2AE0912703A2E241
:101B1000B0E00E946D2AE0912803A3E2B0E00E94A9
:101B20006D2AE0912903A4E2B0E00E946D2AE091C1
:101B30002A03A5E2B0E00E946D2A0E94692AE09182
:101B40000E03A6E2B0E00E946D2AE0E036FCE1E080
:101B5000A7E2B0E00E946D2AE0911003AAE2B0E093
:101B60000E946D2AE98DABE2B0E00E946D2AEB8500
:101B7000FC85A0E4B0E00E94512A0E945027E1E0D9
:101B80004E2E0E94882AA0E0F1FCA1E00E9450297C
:101B9000AE81E4E60E94BB310E94422A51F0689473
:101BA000F1F8EE81EF5FEE83AE81A43611F4E0E050
:101BB000EE83EAE0E61510F4E894F0F80E94232999
:101BC000A0E0F0FCA1E00E945029AE81E0E00E947C
:101BD000B6310E94422A51F06894F0F8EE81E1504B
:101BE000EE83AE81AF3F11F4E3E6EE830E947128ED
:101BF0000E94992AC1F00E949F2AA9F4A09134035F
:101C0000A43119F4E7E0E0933403E0E0E093350316
:101C1000E894F3F8A0913403A33028F0E091340362
:101C2000E150E0933403AB2DEAE00E94CA310E2E5E
:101C30000E94992AC1F00E949F2AA9F4A09134031E
:101C4000A43119F4E7E0E0933403E0E0E0933503D6
:101C5000E894F2F8A0913403A33028F0E091340323
:101C6000E150E0933403AB2D0E94732AAA2DEAE0E1
:101C70000E94CF31E02131F0E0E0E0933503E4E170
:101C8000E0933403EAE0EA1510F4E894F3F80E94D4
:101C900071280E9477280E94AC31E02109F4AEC27D
:101CA0006894F3F8AE81A13049F4A0911503A130F6
:101CB00028F4E0911503EF5FE0931503AE81A230A5
:101CC00049F4A0911603A23328F4E0911603EB5FC8
:101CD000E0931603AE81A33049F4A0911703A43614
:101CE00028F4E0911703EF5FE0931703AE81A4306F
:101CF00049F4A0911903A83228F4E0911903EF5F89
:101D0000E0931903AE81A53031F4AEA1A43618F4E6
:101D1000EEA1EF5FEEA3AE81A63031F4AFA1A43601
:101D200018F4EFA1EF5FEFA3AE81A73031F4A8A5BF
:101D3000A43618F4E8A5EF5FE8A7AE81A83049F40F
:101D4000A0911A03AF3F28F4E0911A03EF5FE093EC
:101D50001A03AE81AC3049F4A0910E03A03328F4ED
:101D6000E0910E03E45FE0930E03AE81AD3069F4C1
:101D7000A0914203B0914303A433E8E0BE0728F4E6
:101D80000E940D2831960E94D127AE81AE3031F4E9
:101D9000AAA1A43618F4EAA1EB5FEAA3AE81AF30A2
:101DA00031F4ABA1A43618F4EBA1EB5FEBA3AE8149
:101DB000A03131F4ACA1A43618F4ECA1EB5FECA394
:101DC000AE81A13131F4AE8DA83C18F4EE8DEB5FFD
:101DD000EE8FAE81A23131F4AF8DA83C18F4EF8DB7
:101DE000EB5FEF8FAE81A33131F4A8A1A83C18F4CA
:101DF000E8A1EB5FE8A3AE81A43169F4A09152039E
:101E0000B0915303A835E2E0BE0728F40E9487276B
:101E10007E960E94EB27AE81A53189F4A0910E0336
:101E2000EAE0EA9FF001EA5BFF4FAF85B889AE17A1
:101E3000BF0728F4EF85F8893196EF87F88BAE81DC
:101E4000A63149F4A0912C03A13028F4E0912C0391
:101E5000EF5FE0932C03AE81A73149F4A0912E03EC
:101E6000A23328F4E0912E03EF5FE0932E03AE81BE
:101E7000A83149F4A0912D03A13028F4E0912D035D
:101E8000EF5FE0932D03AE81A93181F4A32FEFE042
:101E90000E94AA2A0E94552909F03F5FA32FEEE174
:101EA0000E94AA2A0E94362A09F03F5FAE81AA3119
:101EB00059F40E94B12AAC3BE2E0BE0728F40E942C
:101EC000942A31960E94DD27AE81AB3191F40E94B5
:101ED000C426A73EE3E0BE07E0E08E07E0E09E07F1
:101EE00040F40E948726EF5FFF4F6F4F7F4F0E94A5
:101EF000E227AE81AC3161F4A0E023FCA1E0A13087
:101F000038F4E0E023FCE1E0EF5F0E944C3323F87B
:101F1000AE81AD3169F40E944726AE3DE3E0BE07D5
:101F200038F40E9428263A96E0934A03F0934B0334
:101F3000AE81AE3169F40E945126A835E2E0BE07B9
:101F400038F40E9434263A96E0935603F0935703F0
:101F5000AE81AF3149F4A0910603AA3028F4E09194
:101F60000603EF5FE0930603AE81A03249F4A0912F
:101F70000803AB3028F4E0910803EF5FE093080317
:101F8000AE81A13249F4A0910903AB3028F4E0916D
:101F90000903EF5FE0930903AE81A23249F4A091F7
:101FA0000A03AB3028F4E0910A03EF5FE0930A03E1
:101FB000AE81A33249F4A0910B03AB3028F4E09139
:101FC0000B03EF5FE0930B03AE81A43249F4A091C1
:101FD0000C03AB3028F4E0910C03EF5FE0930C03AB
:101FE000AE81A53249F4A0912303A13028F4E091F9
:101FF0002303EF5FE0932303AE81A63249F4A0915F
:102000002403A13028F4E0912403EF5FE09324033C
:10201000AE81A73249F4A0912503A13028F4E091C4
:102020002503EF5FE0932503AE81A83249F4A09128
:102030002603A13028F4E0912603EF5FE093260306
:10204000AE81A93249F4A0912703A13028F4E09190
:102050002703EF5FE0932703AE81AA3249F4A091F2
:102060002803A33028F4E0912803EF5FE0932803CE
:10207000AE81AB3249F4A0912903A13028F4E0915C
:102080002903EF5FE0932903AE81AC3249F4A091BC
:102090002A03A13028F4E0912A03EF5FE0932A039A
:1020A000AE81AD3291F40E945627AF39E6E8BE0703
:1020B000E1E08E07E0E09E0740F40E943E27E65FE5
:1020C000FF4F6F4F7F4F0E944727AE81AE3259F4CA
:1020D0000E94B62AA031E7E2BE0728F40E94A82693
:1020E0003A960E94AD26AE81AF3261F4A0E036FC94
:1020F000A1E0A13038F4E0E036FCE1E0EF5F0E94BF
:102100004C3336F8AE81A03349F4A0911003A130CE
:1021100028F4E0911003EF5FE0931003AE81A13348
:1021200031F4A98DA13018F4E98DEF5FE98FAE810C
:10213000A23359F4AB85BC85A632E2E0BE0728F491
:10214000EB85FC853196EB87FC87AE81AC3549F495
:10215000A0910503AA3F28F4E0910503EB5FE0930B
:102160000503AE81AD3531F4ABA5A73018F4EBA56E
:10217000EF5FEBA7AE81AE3559F4AB89BC89A83BC4
:10218000EBE0BE0728F4EB89FC893196EB8BFC8BE6
:10219000AE81AF3531F4AAA5AA3018F4EAA5EF5FF5
:1021A000EAA7AE81A03631F4A9A5AA3018F4E9A5B2
:1021B000EF5FE9A7AE81A13649F4A0911F03AC33CC
:1021C00028F4E0911F03EF5FE0931F03AE81A23676
:1021D00049F4A0911C03AA3F28F4E0911C03E65F98
:1021E000E0931C03AE81A33649F4A0911B03AA3FE0
:1021F00028F4E0911B03E65FE0931B03EAE0EB1594
:1022000010F4E894F2F8AB2DEAE00E94CA310E2EE9
:10221000A0E0F2FCA1E00E9450290E94992A09F452
:1022200096C26894F2F8AE81A13049F4A0911503EA
:10223000A13028F0E0911503E150E0931503AE8141
:10224000A23049F4A0911603AB3028F0E0911603B8
:10225000E550E0931603AE81A33049F4A091170333
:10226000AD3328F0E0911703E150E0931703AE81FE
:10227000A43049F4A0911903A53128F0E091190385
:10228000E150E0931903AE81A53031F4AEA1A13045
:1022900018F0EEA1E150EEA3AE81A63031F4AFA16B
:1022A000A13018F0EFA1E150EFA3AE81A73031F4D7
:1022B000A8A5A13018F0E8A5E150E8A7AE81A830A4
:1022C00049F4A0911A03A13028F0E0911A03E150DB
:1022D000E0931A03AE81AC3049F4A0910E03A9310A
:1022E00028F0E0910E03EC50E0930E03AE81AD3088
:1022F00069F4A0914203B0914303AD36E7E0BE0715
:1023000028F00E940D2831970E94D127AE81AE306F
:1023100031F4AAA1A63018F0EAA1E550EAA3AE81F3
:10232000AF3031F4ABA1A63018F0EBA1E550EBA330
:10233000AE81A03131F4ACA1A63018F0ECA1E5508B
:10234000ECA3AE81A13131F4AE8DA13018F0EE8D49
:10235000E550EE8FAE81A23131F4AF8DA13018F08F
:10236000EF8DE550EF8FAE81A33131F4A8A1A130FC
:1023700018F0E8A1E550E8A3AE81A43161F4A09182
:102380005203B09153030E94383328F40E948727E8
:102390007E970E94EB27AE81A53189F4A0910E03B0
:1023A000EAE0EA9FF001E654F040AF85B889EA1709
:1023B000FB0728F4EF85F8893197EF87F88BAE811A
:1023C000A63149F4A0912C03A13028F0E0912C0310
:1023D000E150E0932C03AE81A73149F4A0912E0384
:1023E000A23028F0E0912E03E150E0932E03AE815D
:1023F000A83149F4A0912D03A13028F0E0912D03DC
:10240000E150E0932D03AE81A93119F4323008F088
:102410003150AE81AA3159F40E94B12AA935E2E0C7
:10242000BE0728F00E94942A31970E94DD27AE81D2
:10243000AB3191F40E94C426AB30E0E0BE07E0E08F
:102440008E07E0E09E0740F00E948726E150F040B2
:10245000604070400E94E227AE81AC3159F4A0E0A8
:1024600023FCA1E0A13030F0A0E023FCA1E00E9419
:10247000BB2A23F8AE81AD3161F40E9447260E9449
:10248000383338F40E9428263197E0934A03F093BA
:102490004B03AE81AE3161F40E9451260E94383365
:1024A00038F40E9434263197E0935603F093570393
:1024B000AE81AF3149F4A0910603A23028F0E0913B
:1024C0000603E150E0930603AE81A03249F4A091E7
:1024D0000803A23028F0E0910803E150E0930803DC
:1024E000AE81A13249F4A0910903A13028F0E09116
:1024F0000903E150E0930903AE81A23249F4A091AF
:102500000A03A13028F0E0910A03E150E0930A03A6
:10251000AE81A33249F4A0910B03A13028F0E091E1
:102520000B03E150E0930B03AE81A43249F4A09178
:102530000C03A13028F0E0910C03E150E0930C0370
:10254000AE81A53249F4A0912303A13028F0E09197
:102550002303E150E0932303AE81A63249F4A09116
:102560002403A13028F0E0912403E150E0932403F8
:10257000AE81A73249F4A0912503A13028F0E09163
:102580002503E150E0932503AE81A83249F4A091E0
:102590002603A13028F0E0912603E150E0932603C2
:1025A000AE81A93249F4A0912703A13028F0E0912F
:1025B0002703E150E0932703AE81AA3249F4A091AA
:1025C0002803A13028F0E0912803E150E09328038C
:1025D000AE81AB3249F4A0912903A13028F0E091FB
:1025E0002903E150E0932903AE81AC3249F4A09174
:1025F0002A03A13028F0E0912A03E150E0932A0356
:10260000AE81AD3269F40E9456270E943C3340F4FB
:102610000E943E27E150F040604070400E944727F2
:10262000AE81AE3251F40E94B62A0E94383328F4AB
:102630000E94A82631970E94AD26AE81AF3259F490
:10264000A0E036FCA1E0A13030F0A0E036FCA1E033
:102650000E94BB2A36F8AE81A03349F4A091100342
:10266000A13028F0E0911003E150E0931003AE8117
:10267000A13331F4A98DA13018F0E98DE150E98F33
:10268000AE81A23359F4AB85BC85A93CE0E0BE071E
:1026900028F0EB85FC853197EB87FC87AE81AC3564
:1026A00049F4A0910503A13028F0E0910503E5501D
:1026B000E0930503AE81AD3531F4ABA5A13018F040
:1026C000EBA5E150EBA7AE81AE3559F4AB89BC89DF
:1026D000A13DE7E0BE0728F0EB89FC893197EB8B41
:1026E000FC8BAE81AF3531F4AAA5A13018F0EAA574
:1026F000E150EAA7AE81A03631F4A9A5A13018F0C7
:10270000E9A5E150E9A7AE81A13649F4A0911F03E4
:10271000A13028F0E0911F03E150E0931F03AE8148
:10272000A23649F4A0911C03AB3028F0E0911C03C1
:10273000EA50E0931C03AE81A33649F4A0911B0339
:10274000A13028F0E0911B03EA50E0931B0323FC27
:1027500028C0E0913203ACECB3E0FF27662777276F
:102760000E9423300E94DC320E94C22A0E943C3325
:102770003CF40E94CB2A0E94D42A0E94DB2A09C082
:10278000E0E0E093BC03E093BD03E093BE03E0937D
:10279000BF030E94CB2AA4E7B3E00E94DC260E947C
:1027A000E42A23FE4FC0EF81F8850E94FB290E9496
:1027B000E6320E94E132E0E0F0E060E874E40E947A
:1027C000FB30A0E0B0E48CE995E40E94AD30DF017D
:1027D000CB01EB89FC89662777270E9423300E9472
:1027E000A326DF01CB01E3E3F3E365E872E40E9493
:1027F000FB30E093CC03F093CD036093CE03709352
:10280000CF03A0910F03A13048F4E0E0E093CC03A4
:10281000E093CD03E093CE03E093CF030E94CB2A55
:102820000E94DB2AE0910603A0910703AE1750F047
:102830000E94C22A0E946427A4E7B3E00E94DC261B
:102840000E94E42AA0E0F0FCA1E00E945A29E09155
:102850000603A09107030E94C531E021F9F0A98584
:10286000BA85E0E0F4E0EA1BFB0B0E94FB29DF01E4
:10287000CB01EAE9F9E969E271E40E94FB30DF018A
:10288000CB01E0E0F0E068E571E40E94A326AAE74E
:10289000B3E00E94DC26E0E0E0930703F0915803E8
:1028A000E0E0DF01E0913303F0E0EA0FFB1FACE969
:1028B000B3E00E942D260E94E82AA0E0B0E080E16B
:1028C00092E40E94FB307F936F93FF93EF930E94FB
:1028D000B12A0E94F12AAF91BF918F919F916627F3
:1028E00077270E9423300E94AD30E0939C03F09341
:1028F0009D0360939E0370939F030E94F62AE0E07D
:10290000F0E060E87FE30E9466310E2E0E94F62A16
:10291000E0E0F0E068EC72E40E946031E021E9F070
:102920000E94E82A0E94D42AA4E8B3E00E94EC2F77
:102930000E94DC320E94E82AE093A003F093A103F6
:102940006093A2037093A3030E94F62A0E94642757
:10295000A4E4B3E00E945F2615C0E0E0E0938403A6
:10296000E0938503E0938603E0938703E093A0035D
:10297000E093A103E093A203E093A303E093440355
:10298000E09345030E94E8260E945F270E9466317B
:10299000EF930E94FF2A0E946631AF91EA23C1F1B2
:1029A0000E947526E0E0F0E068EC72E40E94FB30E3
:1029B0000E94C4260E94EB320E94A3260E94012B93
:1029C000A0919803B091990380919A0390919B03F1
:1029D000E0E0F0E064E172E40E94AD30DF01CB01A1
:1029E0000E94FF260E94FB30A0E0B0E080E291E46C
:1029F0000E94AD300E94012BE0919803F091990361
:102A000060919A0370919B03DE0114960E94DC266C
:102A10000E942329A0911D03EDEF0E94CA310E22CE
:102A20000E942929E02129F0E0911D03EF5FE09346
:102A30001D03A62D0E94732AA0911D03EFEF0E9493
:102A4000CA310E220E942929E02129F0E894F0F8E9
:102A5000E0E0E0931D03A0911D03EEE10E94AC3184
:102A60000E2E0E942929E02119F0E1E0E0932003D5
:102A7000E0911F03E03019F4E0E0E09320030E94AE
:102A80006D270E945F270E9410320E94492AA09160
:102A900020030E940A2B19F0E1E0E0932003A091AB
:102AA0002003AC3309F41FEFA0910503A13020F0FF
:102AB000E09105030E945B28A0912A030E946E29E1
:102AC000A12F0E940A2B29F1E88DEF5FE88FF0E03B
:102AD0003196BF010E940F2BE617F70784F40E947E
:102AE000162B0E9400320E2E0E94232BE4EAF1E006
:102AF00060E070E00E94F831E02909F010E00E94E7
:102B00000F2BA88DB0E0EA17FB0714F4E0E0E88F84
:102B100002C0E0E0E88FA12F0E9468270E94162BD8
:102B20000E9410320E22AB85BC85E4EAF1E00E94DF
:102B3000DA31E02119F0163908F416E94420C9F415
:102B4000E02FF0E034960E943328AE0FBF1FE12F34
:102B50000E942C2BA4E00E940926A02F0E94362B55
:102B6000A09138030E940926A12F0E9409260E94E5
:102B70003B2BE1E0E41509F057C04424A091170372
:102B80000E94442BE0931803F0E0BC96DF01E09133
:102B90001403F0E0AE0FBF1FE0911503F0E0AE0F9D
:102BA000BF1FE0911603F0E0AE0FBF1FE0911903C5
:102BB000F0E0AE0FBF1FEEA1F0E0AE0FBF1FEFA120
:102BC000F0E0AE0FBF1FE8A5F0E0AE0FBF1FE09131
:102BD0001A030E942C2BACE20E940926A091140338
:102BE0000E940926A09115030E940926A0911603B0
:102BF0000E940926A09118030E940926A09119039A
:102C00000E940926AEA10E940926AFA10E940926B2
:102C1000A8A50E940926A0911A030E94362BA0E0C5
:102C20000E94362B0E943B2B233608F0E4C60E94FC
:102C30008E2A2081A0913003A13048F420FC07C0E7
:102C4000A0E0F799A1E0EA2FE295E07F19C0A0E0AB
:102C5000F799A1E0EA2FE295E07F0E2EA0E0F3992C
:102C6000A1E0EA2FEE0FEE0F0E0EA0E0F499A1E026
:102C7000EA2FEE0FA02DAE0FE0E0F599E1E0EA0FAC
:102C8000ECA7EAE00E944A2BEAE0DE01AE5BBF4F10
:102C9000EC930E944F2BDE01AC5BBF4FEC93EAE05C
:102CA0000E94552BEAE00E945A2BEAE00E945F2B1B
:102CB0000E94642BE89435F8A0E031FCA1E00E946A
:102CC0006E29A0E032FCA1E0E1E00E94AC310E2AC6
:102CD000A0E034FCA1E0E1E00E94AC31E02911F079
:102CE00020FA01C0E894F5F8E0912803E03021F4DF
:102CF0000E94862B0E94972BA0912803A13081F47B
:102D0000A0E022FCA1E0EA2FEE0FE75F0E2EA0E08C
:102D100022FCA1E0EA2FEE0FEE0FE00D0E94A62BA1
:102D2000A0912803A23099F40E94862BA0E022FCF7
:102D3000A1E0EA2F0E94B62B0E0EA0E022FCA1E03B
:102D4000EA2FE295E07FEE0F0E0E0E94972BA091E6
:102D50002803A33031F4E0E022FCE1E0E85F0E94C8
:102D6000A62BA0910E03A83109F041C00E94BB2BF5
:102D7000A23DE0E0BE07E0E08E07E0E09E071CF029
:102D8000E1E0E09301030E94C92BA83FE0E0BE0709
:102D9000E0E08E07E0E09E071CF0E3E0E093010333
:102DA0000E94C92BAF3FE0E0BE07E0E08E07E0E005
:102DB0009E071CF0E7E0E09301030E94C92BA430BA
:102DC000E1E0BE07E0E08E07E0E09E071CF0EFE0E8
:102DD000E09301030E94C92BAE30E1E0BE07E0E0C2
:102DE0008E07E0E09E071CF0EFE1E0930103A09165
:102DF0000E03A43209F041C00E94BB2BA633E1E0D0
:102E0000BE07E0E08E07E0E09E071CF0E1E0E09303
:102E100001030E94C92BAA34E1E0BE07E0E08E075F
:102E2000E0E09E071CF0E3E0E09301030E94C92B61
:102E3000AE35E1E0BE07E0E08E07E0E09E071CF063
:102E4000E7E0E09301030E94C92BA836E1E0BE074A
:102E5000E0E08E07E0E09E071CF0EFE0E093010366
:102E60000E94C92BAC37E1E0BE07E0E08E07E0E04E
:102E70009E071CF0EFE1E0930103A0910E03A03345
:102E800009F041C00E94BB2BA638E1E0BE07E0E09C
:102E90008E07E0E09E071CF0E1E0E09301030E9452
:102EA000C92BAC3CE1E0BE07E0E08E07E0E09E0706
:102EB0001CF0E3E0E09301030E94C92BA63DE1E092
:102EC000BE07E0E08E07E0E09E071CF0E7E0E0933D
:102ED00001030E94C92BA03EE1E0BE07E0E08E079F
:102EE000E0E09E071CF0EFE0E09301030E94C92B95
:102EF000AF3EE1E0BE07E0E08E07E0E09E071CF099
:102F0000EFE1E0930103A0910203A431F0F40E94E9
:102F10006D270E94D22B6CF0FE01E05CFF4F3396D0
:102F2000FF93EF930E94DA2B0E94E02BAF91BF91A9
:102F3000EC930E94EB2BFF93EF930E94DA2B0E94FD
:102F4000A732AF91BF91EC930DC020FE05C0E0E425
:102F50000E94F02BE0E402C00E944F2BDE01AC5B2C
:102F6000BF4FEC93AF89A13050F0EF89E150EF8B68
:102F7000E8E70E94F02BFE01E05CFF4F0483AE897E
:102F8000A13058F0EE89E150EE8BE8E30E94F02B7F
:102F90000E94EB2BA0912B03A083AD89A13058F0A8
:102FA000ED89E150ED8BE9E30E94F02BE0E5DE01D5
:102FB000AC5BBF4FEC93E0911103E03009F5EDA558
:102FC000E058EDA7A0917503AA2382F4E0E40E94E3
:102FD0004A2BA0917403B0917503AD39EFEFBE0792
:102FE00014F4689435F80E94F52B02C0E89435F883
:102FF0000E94052C1A9714F00E940A2C0E941C2C87
:10300000A0911103A13009F046C0ECA5E85FECA740
:10301000A0917B03AA23A2F4E0E40E944A2B0E9421
:10302000292CA73FEFEFBE0714F4689401C0E89481
:1030300035F8E0917A03F0917B030E94763106C067
:10304000E89435F8E0917A03F0917B03E0937603FE
:10305000F09377030E94052C1A9714F00E940A2C13
:103060000E941C2C0E94292CE3E6F0E00E94E6312D
:103070000E2E0E94292CEDE9FFEF0E94E031E0299D
:1030800051F0E89435F8E0E40E944A2BE0E4DE01D8
:10309000AE5BBF4FEC930E942E2CFF93EF930E94E8
:1030A000C92B0E94332C0E94E02BAF91BF910E944C
:1030B000382C3696FF93EF930E943D2C0E94E02B14
:1030C000AF91BF910E94382C3796FF93EF930E94E7
:1030D0003D2C0E94A732AF91BF91EC930E94C92B67
:1030E000A639E0E0BE07E0E08E07E0E09E0764F46A
:1030F000E0E40E94552BE0E40E945A2BE0E40E9499
:103100005F2BE0E0E0930103213009F061C00E94F1
:10311000432C0E944D2CA83EE3E0BE07C8F0EEA56C
:10312000E05EEEA70E94522C0E94582C0E94382C80
:103130003E96BF010E944D2C0E94632C0E94382CA9
:103140003F96BF010E944D2C0E94F12ADF011DC055
:10315000EEA5E056EEA70E944D2CA436E0E0BE0797
:1031600028F00E94522C0E94632CEC930E946E2C3B
:10317000BF010E944D2C0E94F12A0E94732C0E94D4
:10318000382C3F96BF010E944D2CEAE0F0E00E94EF
:103190007A2CA0910003AA3010F00E947F2CFE012F
:1031A000E05CFF4F3996BF01A09100030E94852C7F
:1031B0000E94382C3A96BF01AC2DB0E00E948C2CB6
:1031C0000E94382C3B96BF01AC2D0E94852CEC93BD
:1031D000223009F06FC0EEA5E05CEEA70E945627F2
:1031E000A03AE6E8BE07E1E08E07E0E09E0778F04F
:1031F0000E94972CFF93EF930E945627E0EAF6E88F
:1032000061E070E00E949C2CAF91BF91EC930E9412
:1032100056270E94A72C78F00E94AF2CFF93EF93C3
:103220000E945627E0E1F7E260E070E00E949C2CEB
:10323000AF91BF91EC930E9456270E94B42C68F086
:103240000E94BC2CFF93EF930E9456270E941729DF
:103250000E949C2CAF91BF91EC930E9456270E9434
:10326000C12C68F00E94C92CFF93EF930E9456274F
:103270000E94332C0E949C2CAF91BF91EC930E9432
:1032800056270E94D22B58F00E946E2CFF93EF938A
:103290000E94CE2C0E949C2CAF91BF91EC930E9477
:1032A000D42CFF93EF930E94CE2C0E94A332AF91B7
:1032B000BF91EC93233009F08DC0E7E70E94D92C31
:1032C000A0919303AA2392F4E0919003F0919103CB
:1032D00060919203709193030E947A31E09390037E
:1032E000F093910360939203709393030E94FF2ADB
:1032F0000E94A326772312F40E94E32C0E94FF2A47
:103300000E94A3260E94E92C10F40E94F22C0E9435
:10331000FF2A0E94A3260E94F82C10F40E94012D7F
:103320000E94FF2A0E94A3260E94072D10F40E94EB
:103330000A2D0E94102D0E94A72C7CF00E94AF2C19
:10334000FF93EF930E94102DE0E1F7E260E070E060
:103350000E94E02BAF91BF91EC930E94102D0E9430
:10336000B42C6CF00E94BC2CFF93EF930E94102DA4
:103370000E9417290E94E02BAF91BF91EC930E940D
:10338000102D0E94C12C5CF00E94C92CFF93EF937A
:103390000E94102D0E94192DAF91BF91EC930E94B5
:1033A000102D0E94D22B5CF00E946E2CFF93EF93A5
:1033B0000E941B2D0E94E02BAF91BF91EC930E94C5
:1033C000D42CFF93EF930E941B2D0E94A732AF9144
:1033D000BF91EC93243009F051C00E94212DA0919F
:1033E0007103AA2312F40E94262D0E94312D772307
:1033F00012F40E94E32C0E94312D0E94E92C10F45B
:103400000E94F22C0E94312D0E94F82C10F40E9490
:10341000012D0E94312D0E94072D10F40E940A2DCB
:103420000E94372DA031E7E2BE0724F00E94AF2CA6
:103430000E943C2D0E94372DA83EE3E0BE0724F0F9
:103440000E94BC2C0E944A2D0E94372DA436E0E039
:10345000BE0724F00E94C92C0E94582D0E94372DCF
:103460001A9744F00E946E2CBF010E94372D0E94D3
:103470008C2CEC930E94D42C0E94662D253051F5A3
:103480000E94212D0E946F2DA091C303AA2312F444
:103490000E94F22C0E94E826E0E0F0E066EC72EC7C
:1034A0000E94403110F40E94012D0E94752DA43617
:1034B000E0E0BE0724F00E94C92C0E947A2D0E94F1
:1034C0006E2CBF010E94752D0E948C2C0E94382CFE
:1034D0000E94882D2630D9F5EEA5E058EEA7E0E051
:1034E0000E94922DE5E00E94972DE8E70E949C2D16
:1034F000AC81BD81A83EE3E0BE074CF00E94BC2C2D
:10350000BF01AC81BD81E8EEF3E00E94A12DAC814A
:10351000BD81A436E0E0BE074CF00E94C92CBF017B
:10352000AC81BD81E4E6F0E00E94A12D0E946E2CEA
:10353000BF01AC81BD810E948C2C0E94382C3F962B
:10354000BF01AC81BD810E94AB2DDB01EC93273024
:1035500009F05AC0113058F1ECE00E94922DA12FD1
:103560000E94442BE436A0E0FA074CF00E94972C0E
:10357000BF01A12FB0E0E8ECF0E00E94A12DA12F47
:103580000E94442B3A974CF00E94AF2CBF01A12F10
:10359000B0E0E4E1F0E00E94A12D0E94BC2CBF014C
:1035A000A12F0E94442BDF010E94AB2D2BC0EBE02A
:1035B0000E94922D0E94B02DE436A0E0FA0750F050
:1035C0000E94972CBF01AD85BE85E8ECF0E00E941B
:1035D000B52DEC930E94B02D3A9750F00E94AF2C7D
:1035E000BF01AD85BE85E4E1F0E00E94B52DEC930E
:1035F0000E94BC2CBF010E94B02DDF01EAE0F0E088
:103600000E949232DB01EC93283009F081C00E94C5
:10361000432CA0916C03B0916D03A135EBEFBE0775
:1036200034F4E1E5FBEFE0936C03F0936D03A091BC
:103630006C03B0916D03A03BE4E0BE0734F0EFEA09
:10364000F4E0E0936C03F0936D03A0916D03AA2363
:103650004AF40E94012DE0916C03F0916D030E94E9
:10366000763104C0E0916C03F0916D03E0936E033A
:10367000F0936F03A0916E03B0916F03ECE3F0E061
:103680000E946332E0934C03F0934D030E94B82DE7
:10369000ECE30E944032A0916E03B0916F03AE1B29
:1036A000BF0BA0934E03B0934F0324FE28C00E948B
:1036B000B82D1A9710F00E947F2CFE01E05CFF4F9E
:1036C0003996BF010E94B82DEAE0F0E00E949232E4
:1036D000DB010E94382C3A96BF01A0914E03B091B5
:1036E0004F030E94F12A0E94732C0E94382C3B96B3
:1036F000BF01A0914E03B0914F030E94BD2DE3E79F
:103700000E94C02DE8E30E94C52DE4E50E94CA2D69
:10371000293009F057C0EEA5E058EEA70E947F2C93
:10372000EEE30E94D92CA0917103AA2312F40E9407
:10373000262D0E94312D772312F40E94E32C0E9443
:10374000312D0E94E92C10F40E94F22C0E94312DA0
:103750000E94F82C10F40E94012D0E94312D0E942D
:10376000072D10F40E940A2D0E94372DA031E7E2A8
:10377000BE0724F00E94AF2C0E943C2D0E94372DE2
:10378000A83EE3E0BE0724F00E94BC2C0E944A2D14
:103790000E94372DA436E0E0BE0724F00E94C92C19
:1037A0000E94582D0E94372D1A9744F00E946E2CCB
:1037B000BF010E94372D0E948C2CEC930E94D42CC8
:1037C0000E94662D2A30F9F4EEA5E058EEA70E947B
:1037D0007F2CEEE30E94D92C0E946F2D0E94752D44
:1037E000A436E0E0BE0724F00E94C92C0E947A2D86
:1037F0000E946E2CBF010E94752D0E948C2C0E948D
:10380000382C0E94882D2B3091F5EEA5E054EEA7C0
:103810000E94CF2D0E94B62AA83EE3E0BE0740F0EA
:103820000E94BC2CBF010E94B62A0E94582CEC9327
:103830000E94B62AA436E0E0BE0740F00E94C92CE0
:10384000BF010E94B62A0E94632CEC930E946E2C4A
:10385000BF010E94B62A0E94F12A0E94732C0E9486
:10386000382C3F96BF010E94B62A0E94BD2DAC8D18
:103870000E946827AB8DE0E00E94CF31E02909F477
:10388000B3C0EEA5EF77EEA7E0913103E170EE0F44
:10389000ADA5EA23EDA7E0913103E6950E94D32D73
:1038A0000E2EE0913103E695E695E170AE2FE0E053
:1038B000F5FCE1E0EA2BEE0FEE0FE00DADA5EA0F0F
:1038C000EDA70E94642BAB8D0E946827AC8D0E94EF
:1038D0000A2B49F1AB8DA13021F40E94D82D0E9412
:1038E000DB2DAB8DA23029F40E94D82DEDE00E9493
:1038F000E12DAB8DA33029F40E94D82DEBE00E947E
:10390000E12D0E94E62D21F00E94D82D0E94DB2D92
:103910000E946C280E94F02D29F00E94D82DEBE027
:103920000E94E12D2AC0AB8DA13029F40E94F62D12
:10393000ECE00E94CA2DAB8DA23029F40E94F62D36
:10394000EDE00E94CA2DAB8DA33029F40E94F62D24
:10395000EBE00E94CA2D0E94E62D29F00E94F62D70
:10396000ECE00E94CA2D0E946C280E94F02D29F0E4
:103970000E94F62DEBE00E94CA2DAC8DA13029F4F7
:103980000E94FA2DECE00E94CA2DAC8DA23029F4E1
:103990000E94FA2DEDE00E94CA2DAC8DA33029F4CF
:1039A0000E94FA2DEBE00E94CA2DAC8DE4E00E944B
:1039B000AC310E94F02D29F00E94FA2DECE00E941B
:1039C000CA2DAC8DE5E00E94AC310E94F02D29F0AB
:1039D0000E94FA2DEBE00E94CA2DE0911103E03025
:1039E00019F4EDA5E058EDA7F29B05C0EDA5EB7F1E
:1039F000EDA7EF5FEDA7233609F06BC551E050311D
:103A000040F40E94FE2DEAE0EC93E89435F85F5F05
:103A1000F6CFAE81EBE50E94062EEAE50E94AC31BE
:103A2000E02911F0E2E3EE83AE81A33311F4ECE57B
:103A3000EE83EE81E03029F4E0911403F0E0E98BAD
:103A4000FA8BAE81A13029F4E0911503F0E0E98B07
:103A5000FA8BAE81A23029F4E0911603F0E0E98BF5
:103A6000FA8BAE81A33029F4E0911703F0E0E98BE3
:103A7000FA8BAE81A43029F4E0911903F0E0E98BD0
:103A8000FA8BAE81A53021F4EEA1F0E0E98BFA8B40
:103A9000AE81A63021F4EFA1F0E0E98BFA8BAE8184
:103AA000A73021F4E8A5F0E0E98BFA8BAE81A830CD
:103AB00029F4E0911A03F0E0E98BFA8BAE81A9308A
:103AC00019F4E0E0E98BEA8BAE81AA3019F4E0E06A
:103AD000E98BEA8BAE81AB3019F4E0E0E98BEA8B3D
:103AE000AE81AC3029F4E0910E03F0E0E98BFA8B63
:103AF000AE81AD3021F40E940D28E98BFA8BAE81A6
:103B0000AE3021F4EAA1F0E0E98BFA8BAE81AF3060
:103B100021F4EBA1F0E0E98BFA8BAE81A03121F426
:103B2000ECA1F0E0E98BFA8BAE81A13121F4EE8DAE
:103B3000F0E0E98BFA8BAE81A23121F4EF8DF0E059
:103B4000E98BFA8BAE81A33121F4E8A1F0E0E98B97
:103B5000FA8BAE81A43121F40E948727E98BFA8B7E
:103B6000AE81A53121F4EF85F889E98BFA8BAE811E
:103B7000A63129F4E0912C03F0E0E98BFA8BAE81B9
:103B8000A73129F4E0912E03F0E0E98BFA8BAE81A6
:103B9000A83129F4E0912D03F0E0E98BFA8BAE8196
:103BA000A93121F4E32FF0E0E98BFA8BAE81AA3141
:103BB00021F40E94942AE98BFA8BAE81AB3131F467
:103BC000E0916203F0916303E98BFA8BAE81AC3133
:103BD00031F4E0E023FCE1E0F0E0E98BFA8BAE8128
:103BE000AD3121F40E942826E98BFA8BAE81AE31EB
:103BF00021F40E943426E98BFA8BAE81AF3129F48F
:103C0000E0910603F0E0E98BFA8BAE81A03229F453
:103C1000E0910803F0E0E98BFA8BAE81A13229F440
:103C2000E0910903F0E0E98BFA8BAE81A23229F42E
:103C3000E0910A03F0E0E98BFA8BAE81A33229F41C
:103C4000E0910B03F0E0E98BFA8BAE81A43229F40A
:103C5000E0910C03F0E0E98BFA8BAE81A53229F4F8
:103C6000E0912303F0E0E98BFA8BAE81A63229F4D0
:103C7000E0912403F0E0E98BFA8BAE81A73229F4BE
:103C8000E0912503F0E0E98BFA8BAE81A83229F4AC
:103C9000E0912603F0E0E98BFA8BAE81A93229F49A
:103CA000E0912703F0E0E98BFA8BAE81AA3229F488
:103CB000E0912803F0E0E98BFA8BAE81AB3229F476
:103CC000E0912903F0E0E98BFA8BAE81AC3229F464
:103CD000E0912A03F0E0E98BFA8BAE81AD3231F44A
:103CE000E0915E03F0915F03E98BFA8BAE81AE3217
:103CF00021F40E94A826E98BFA8BAE81AF3231F411
:103D0000E0E036FCE1E0F0E0E98BFA8BAE81A03335
:103D100029F4E0911003F0E0E98BFA8BAE81A13336
:103D200021F4E98DF0E0E98BFA8BAE81A23321F426
:103D3000EB85FC85E98BFA8BAE81AC3529F4E091FB
:103D40000503F0E0E98BFA8BAE81AD3521F4EBA5EC
:103D5000F0E0E98BFA8BAE81AE3521F4EB89FC897A
:103D6000E98BFA8BAE81AF3521F4EAA5F0E0E98B5F
:103D7000FA8BAE81A03621F4E9A5F0E0E98BFA8B4D
:103D8000AE81A13629F4E0911F03F0E0E98BFA8BB4
:103D9000AE81A23629F4E0911C03F0E0E98BFA8BA6
:103DA000AE81A33629F4E0911B03F0E0E98BFA8B96
:103DB000AE810E945A29AE81E3E00E940B2EE1E120
:103DC0000E940B2EE2E10E940B2EE3E10E940B2EDB
:103DD000E5E10E940B2EEBE10E940B2EEDE10E942B
:103DE0000B2EEEE20E94AC31E0291E2E0E94102E16
:103DF0000E94DA31E021E12911F0F69A01C0F6982B
:103E0000A0E0F699A1E0EA2FE795E0E0E795EEA7BC
:103E1000E0E0EDA7ECA7E0930103FE01E05CFF4FBB
:103E20003396BF01AE81B0E0A7FDBFEF0E948C2C9E
:103E3000EC930E94EB2BBF01AE81B0E0A7FDBFEF7A
:103E40000E94AB2DDB01EC93A989BA89A031E7E28E
:103E5000BE0750F00E94AF2CBF01A989BA89E0E1EA
:103E6000F7E20E94B52DEC93A989BA89A83EE3E058
:103E7000BE0740F00E94BC2CBF01A989BA890E94EC
:103E8000582CEC93A989BA89A436E0E0BE0740F02B
:103E90000E94C92CBF01A989BA890E94632CEC93A6
:103EA000A989BA891A9738F00E946E2C0E941A2E9E
:103EB0000E94732CEC930E94D42CBF01A989BA896B
:103EC0000E94BD2DEE81E03091F4EDE60E94552B6D
:103ED000E9E70E945A2BE8E70E945F2BEDE60E947B
:103EE000972DE4E50E949C2DE0E50E94E12DAE8136
:103EF000E1E10E94062EE2E10E940B2EE3E10E9426
:103F00000B2EE5E10E940B2EEDE10E940B2EEEE25E
:103F10000E94AC31E02939F00E946E2C0E941A2ECA
:103F20000E94732CEC93E7EAE0937A000E94292820
:103F3000E7E2E0937A000E941E2EEEE00E940B2E34
:103F4000E1E10E94AC31E02911F0E1E07E2EAE818A
:103F5000E6E00E94062EEFE00E940B2EE2E10E94B6
:103F6000AC31E02911F0E2E07E2EAE81E7E00E9464
:103F7000062EE0E10E940B2E0E94212E11F0E3E0BC
:103F80007E2E0E943328D39708F453C00E948128C4
:103F90000E948628E72D0E948D2810F00E94A028FC
:103FA000E72D0E94A7280E94262EAC91A13008F48C
:103FB0003FC00E942D2E0E94CB280E9447334CF414
:103FC0000E94262E0E94362E0E946C310E94402EA6
:103FD00023C00E94492E0E94EC28EF930E94492E94
:103FE0000E94F528AF91EA2379F00E94262E0E94C4
:103FF000362E0E947131A0938003B0938103809389
:1040000082039093830308C00E94492E0E94FE28D9
:104010001CF00E944B2E0CC0A0918003B091810334
:1040200080918203909183030E9417290E941C298A
:1040300004C00E9461280E944B2EAE81AD3019F55C
:104040000E942E2CFF93EF930E94232B0E94192D88
:10405000AF91BF910E94382C3696FF93EF930E9448
:104060005A2E0E94E02BAF91BF910E94382C3796B8
:10407000FF93EF930E945A2E0E94A732AF91BF91F7
:10408000EC93E0E2ECA7AE81A53119F50E942E2C4D
:10409000FF93EF930E94232B0E94192DAF91BF91A4
:1040A0000E94382C3696FF93EF930E945A2E0E945E
:1040B000E02BAF91BF910E94382C3796FF93EF937E
:1040C0000E945A2E0E94A732AF91BF91EC93E0E676
:1040D000ECA70E941E2EEEE00E940B2EE1E10E9452
:1040E000AC31E029B1F00E94602EE4E00E94642E21
:1040F00028F00E942E2C0E946A2EEC930E943328F6
:104100001A9728F00E946D2E0E94732CEC930E9447
:10411000742EAE81E6E00E94062EEFE00E940B2E88
:10412000E2E10E94AC31E029B1F00E94602EE2E0B1
:104130000E94642E28F00E942E2C0E946A2EEC937E
:104140000E9433281A9728F00E946D2E0E94732C2B
:10415000EC930E94742EAE81E7E00E94062EE0E10F
:104160000E940B2E0E94212EB1F00E94602EE1E0F1
:104170000E94642E28F00E942E2C0E946A2EEC933E
:104180000E9433281A9728F00E946D2E0E94732CEB
:10419000EC930E94742EAE81A431B1F40E942E2CB7
:1041A0000E947B2E0E94632C0E94382C36960E941F
:1041B0007B2E0E94F12A0E94732C0E94382C379685
:1041C0000E947B2E0E94BD2DAE81A63129F40E9453
:1041D000812EEBE00E94E12DAE81A73121F40E94F7
:1041E000812E0E94012DAE81A83121F40E94812EE2
:1041F0000E94DB2DAE81A931D1F4A091CF03AA2377
:1042000012F40E94F52B0E942E2CBF010E94052C57
:104210000E948C2C0E94382C3696BF010E94052CDF
:104220000E94AB2DDB01EC93E7E70E945F2BAE8190
:10423000AA31B1F40E942E2C0E94872E0E94632C7A
:104240000E94382C36960E94872E0E94F12A0E94E6
:10425000732C0E94382C37960E94872E0E94BD2D09
:10426000AE81AB3181F4ECE70E94922DE7E70E942A
:10427000972DE8E70E949C2D0E946E2C0E941A2E1A
:104280000E94732CEC93AE81EDE10E94062EEEE1CC
:104290000E94AC31E02939F1E3E70E94922DE8E376
:1042A0000E94972DAE81AD3111F4EEE501C0E8E733
:1042B000DE01A55BBF4FEC930E948D2E1A9760F034
:1042C000FE01E05CFF4F3696BF010E948D2E0E94DA
:1042D000F12A0E94732CEC930E94922EBF010E943F
:1042E0008D2E0E94BD2D0E941E2EE6E00E940B2EF8
:1042F000E7E00E94AC31E02919F0E3E70E94922D3B
:10430000AE81EEE00E94062EEFE00E940B2EE0E16F
:104310000E94AC31E02949F0EDE60E94922DE9E7D8
:104320000E94972DE4E50E949C2DAE81E1E10E9460
:10433000062EE2E10E940B2E0E94212E19F0E8E7E2
:104340000E94972DAE81EFE10E94C0310E2EE5E272
:104350000E94BB31E02161F0EDE60E94552BE8E5BB
:104360000E945A2B0E94922EDF01EE81EF51EC93B6
:10437000AE81AD3219F4EEA5E05CEEA7AE81AE32AF
:1043800011F40E94CF2D0E94102E0E94D431E02102
:1043900049F0E0E00E94C02DE1E70E94C52DE1E771
:1043A0000E94CA2DAE81AD3509F03EC0E7E70E94FC
:1043B000E12DEEE50E94C02DE9E30E94C52D0E948B
:1043C000D42CABA5A083E7EAE0937A000E94F427FF
:1043D000E0933A03F0933B03E7E2E0937A000E9414
:1043E000972EA436E0E0BE0740F00E942E2CBF01BD
:1043F0000E94972E0E94632CEC930E94972E1A978E
:1044000060F0FE01E05CFF4F3696BF010E94972EE0
:104410000E94F12A0E94732CEC930E94922EBF01FD
:104420000E94972E0E94BD2DAE81AE35D9F50E9417
:10443000C22A0E946427A6E7B3E00E94DC26A0916E
:10444000CF03AA2352F4E0917603F09177030E9400
:104450007631E0937603F09377030E942E2CBF0110
:104460000E94052CE4E6F0E00E946332DF010E9426
:10447000AB2DDB010E94382C3696BF010E94052C23
:104480000E948C2C0E94382C3796BF010E94052C6C
:104490000E94AB2DDB01EC93EEE50E94922DE1E052
:1044A0000E94972DAE81AF3531F4EEE50E94922D3A
:1044B000E2E00E94972DAE81A03631F4EEE50E9435
:1044C000922DE3E00E94972DAE81A23611F4E0E137
:1044D000ECA751E0503108F089C00E94FE2DEC910C
:1044E000E03021F40E94FE2DEFE3EC930E94FE2DBC
:1044F000AC91A63021F40E94FE2DEDE7EC930E94D2
:10450000FE2DAC91A13021F40E94FE2DE6E0EC934B
:104510000E94FE2DAC91A23021F40E94FE2DEBE50D
:10452000EC930E94FE2DAC91A33021F40E94FE2D4D
:10453000EFE4EC930E94FE2DAC91A43021F40E9494
:10454000FE2DE6E6EC930E94FE2DAC91A53021F401
:104550000E94FE2DEDE6EC930E94FE2DAC91A7305B
:1045600021F40E94FE2DE7E0EC930E94FE2DAC9119
:10457000A83021F40E94FE2DEFE7EC930E94FE2D5F
:10458000AC91A93021F40E94FE2DEFE6EC930E943D
:10459000FE2DAC91AA3021F40E94FE2DE0E0EC93B8
:1045A0000E94FE2DAC91AB3021F40E94FE2DE1E083
:1045B000EC930E94FE2DAC91AC3021F40E94FE2DB4
:1045C000E8E0EC930E94FE2DAC91AD3021F40E9406
:1045D000FE2DE0E4EC930E94FE2DAC91AE3021F470
:1045E0000E94FE2DE9E0EC935F5F74CFE091010340
:1045F000E695E6950E949C2E0E94A22E0E94A72E70
:104600000E94A22E0E94AF2E0E94A22E0E94BA2EBD
:104610000E94A22E0E94D32D0E94C12E0E94C42E61
:104620000E94C12E0E94C92E0E94C12E0E94CE2E31
:10463000E8ABE0910103E695E695E6950E949C2E95
:104640000E94D42E0E94A72E0E94D42E0E94AF2E2C
:104650000E94D42E0E94BA2E0E94D92E0E94D32DE1
:104660000E94DE2E0E94C42E0E94DE2E0E94C92EC1
:104670000E94DE2E0E94CE2EE9ABE0910103E6956A
:104680000E949C2E0E94D92E0E94A72E0E94D92EF5
:104690000E94AF2E0E94D92E0E94BA2E0E94D42EC4
:1046A0000E94D32D0E94E12E0E94C42E0E94E12E72
:1046B0000E94C92E0E94E12E0E94CE2EEAABFE017E
:1046C000E85BFF4FE0810E949C2E0E94E42E0E9436
:1046D000A72E0E94E42E0E94AF2E0E94E42E0E947C
:1046E000BA2EEEA50E94D32DEA2BAE2FEEA50E9486
:1046F000C42EEA2BAE2FEEA50E94C92EEA2BAE2FB8
:10470000E0910103E170EA2BEBAB0E94E92E0E94DD
:104710009C2E0E94E92E0E94EE2E0E94E92E0E94FD
:10472000F42E0E94E92E0E94FD2E0E94072F0E9467
:104730000B2F0E940E2F0E940B2F0E94152F0E94FC
:104740000B2FE295E170EA2BECAB0E941C2F0E942C
:104750009C2E0E941C2F0E94EE2E0E941C2F0E9455
:10476000F42E0E941C2F0E94FD2EE2950E94D32D54
:104770000E94212F0E940E2F0E94212F0E94152F90
:104780000E94212FE295E170EA2BEDABEEA50E948D
:10479000282F0E941C2F0E94A72E0E941C2F0E94CF
:1047A000AF2E0E941C2F0E94BA2E0E942C2F0E9416
:1047B000D32D0E94312F0E94C42E0E94312F0E94BF
:1047C000C92E0E94312F0E94CE2EEEAB0E94342FB4
:1047D0000E949C2E0E94342F0E94EE2E0E94342FA5
:1047E0000E94F42E0E94342F0E94FD2E0E94392F29
:1047F0000E94D32D0E94312F0E940E2F0E94312F34
:104800000E94152F0E94312FE295E170EA2BEFAB49
:104810000E943E2F0E949C2E0E943E2F0E94EE2E50
:104820000E943E2F0E94F42E0E943E2F0E94FD2ED9
:10483000EE1FE0E0EE1F0E94D32D0E94432F0E9446
:104840000E2F0E94432F0E94152F0E94432FE295A6
:10485000E170EA2BE8AFEDA5E2950E949C2E0E9444
:104860003E2F0E94A72E0E943E2F0E94AF2E0E9434
:104870003E2F0E94BA2E0E94E42E0E94D32D0E9449
:104880004A2F0E94C42E0E944A2F0E94C92E0E94C5
:104890004A2F0E94CE2EE9AF0E944D2F0E949C2EDF
:1048A0000E944D2F0E94EE2E0E944D2F0E94F42E4A
:1048B0000E944D2FE695E695E6950E94522F0E2E0A
:1048C000A0E035FCA1E0EA2FEE0FEE0FEE0FE0299D
:1048D0000E94572FE2950E945D2F0E94572F0E9441
:1048E000152FEA2B0E94572FE295EF70E695E170A5
:1048F000EA2BEAAFFE01EF5BFF4FE081E695E6951C
:10490000E6950E949C2EFE01EF5BFF4FE081E6954D
:10491000E6950E94622F0E94572F0E94662F0E94E8
:10492000572F0E94522FAE2FEDA50E94072FEA2B82
:10493000AE2FEDA50E946D2FAE2FEDA50E94702F1A
:10494000EDA5E695E170EA2BEBAFEDA50E94282FCF
:104950000E94752FE2950E94622FAE2F0E94752F44
:104960000E94AF2E0E94752F0E947A2FAE2F0E94B8
:10497000752F0E94072FEA2BAE2F0E94752F0E94E1
:104980006D2FAE2F0E94752FE6950E94702F0E940A
:10499000752FE170EA2BECAFEDA50E94392F0E9434
:1049A0009C2EECA50E94622FAE2FECA50E94662FD4
:1049B000AE2FECA5E695E6950E94522FAE2FE09122
:1049C0000103E2950E94D32DEA2BAE2FEDA5EE1F39
:1049D000E0E0EE1F0E945D2FAE2FECA5E695E69578
:1049E000E6950E94702FECA5E295E170EA2BEDAF01
:1049F000ECA50E94282F0E947E2FE2950E94622F34
:104A0000AE2F0E947E2F0E94AF2E0E947E2F0E940A
:104A10007A2F0E94832F0E94072FEA2B0E94832F58
:104A20000E946D2F0E94832FE6950E94702F0E9496
:104A3000892FE170EA2BEEAFECA50E94392F0E947E
:104A40009C2E0E94892FE2950E94622F0E94832F44
:104A50000E94AF2E0E94892F0E947A2FAE2F0E94B3
:104A60007E2F0E94072FEA2BAE2F0E947E2F0E94DE
:104A70006D2FAE2F0E947E2FE6950E94702F0E9410
:104A80007E2FE170EA2BEFAF33FE0DC051E05131C4
:104A900050F4E52FF0E0DE019F96AE0FBF1FEFEF61
:104AA000EC935F5FF4CF0E948E2F5D3078F40E940C
:104AB000942FA2E5B8E00E948A31E17011F45D986C
:104AC00001C05D9A0E949B2F5F5FEFCF0E94A32FD2
:104AD0005D3078F40E94942FA0E3B8E00E948A3100
:104AE000E17011F45D9801C05D9A0E949B2F5F5F99
:104AF000EFCF0E94A32F5D3078F40E94942FA2E0A4
:104B0000B8E00E948A31E17011F45D9801C05D9AAD
:104B10000E949B2F5F5FEFCF0E94A32F5D3078F440
:104B20000E94942FA6E0B8E00E948A31E17011F44F
:104B30005D9801C05D9A0E949B2F5F5FEFCF0E943E
:104B4000A32F5A3098F45E9885E28A95F1F7E9E050
:104B5000E51BA0E4B1E00E948A31E17011F45D9898
:104B600001C05D9A0E949B2F5F5FEBCF41E0413116
:104B7000E8F451E05930C0F45E9885E28A95F1F787
:104B8000E42FF0E0DE019F96AE0FBF1FAC91E8E08E
:104B9000E51B0E948231E17011F45D9801C05D9ABD
:104BA0000E949B2F5F5FE6CF4F5FE1CF5D9A85E26A
:104BB0008A95F1F7289A8DEC9AE00197F1F70E9417
:104BC0002329A92DEAE00E94CA310E2AAB2DEAE082
:104BD0000E94CA310E2AAA2DEAE00E94CA31E029B9
:104BE00029F0E0E0E0935403E0935503A82DE4E6B8
:104BF0000E94CF310E2EA0E0F099A1E00E9455292D
:104C000029F00E948C27F09AE89433F80C94D90587
:104C1000FFCFAA93E091C000E072E1F3E881E09356
:104C2000C60021960895A0913E03B0913F030895D8
:104C3000A091A003B091A1038091A2039091A3033E
:104C40000895E0E0F0E061EE75E40E94FB30089525
:104C5000E0914A03F0914B030895662777270E945D
:104C600023300E94DC320895E0915603F0915703FF
:104C70000895A091A803B091A9038091AA039091EF
:104C8000AB030895E0E0F0E060E271E40895A091E4
:104C90004A03B0914B030895E0E0F0E00E94F23146
:104CA0000895A0915603B09157030895E091D00361
:104CB000F091D1036091D2037091D30308950E94C3
:104CC000EA2FED93FC930895A091BC03B091BD032E
:104CD0008091BE039091BF03E0E0F0E06AE774E4E6
:104CE0000E94AD30DF01CB01ACCFA091B803B091F1
:104CF000B9038091BA039091BB030895A091DC039E
:104D0000B091DD038091DE039091DF030895E0917F
:104D10006203F091630360916403709165030895E9
:104D2000A4E6B0E080E090E00E942032DF01CB01F9
:104D3000E091B803F091B9036091BA037091BB039D
:104D40000E94EB3208950E94F0320E94563008957E
:104D5000E0915C03F0915D030895E0935C03F093B0
:104D60005D030895A091D803B091D9038091DA032F
:104D70009091DB030895E093D803F093D9036093F7
:104D8000DA037093DB030895A0916203B09163038B
:104D9000809164039091650308950E942032DF01A1
:104DA000CB01E091D803F091D9036091DA037091BF
:104DB000DB030E94EB32C7CF0E94EC2FED93FC93F4
:104DC0000895E0E0F0E061EE75E40E94AD300895F2
:104DD000A091C003B091C1038091C2039091C3031D
:104DE0000895E0E0F0EC69E774EC0E94403108952A
:104DF000E7EEF3E0E0937803F09379030895E09110
:104E0000C003F091C1036091C2037091C303089580
:104E1000E091C403F091C5036091C6037091C7038C
:104E20000895A091A403B091A5038091A603909149
:104E3000A7030895E093A403F093A5036093A6034A
:104E40007093A7030895A091AC03B091AD03809136
:104E5000AE039091AF030895E091A403F091A503F0
:104E60006091A6037091A7030895A091B403B09137
:104E7000B5038091B6039091B7030895E0915E0366
:104E8000F0915F0360916003709161030895E09376
:104E90005E03F0935F036093600370936103089572
:104EA000EDDFA2E4B0E00E9411330895A0915E030B
:104EB000B0915F0380916003909161030895E0E0F9
:104EC000F0E060E070E00895DDDE0E94AD3008950E
:104ED000E0E00E94CF310E2E0895A0918403B0919E
:104EE0008503809186039091870308950E22A091F7
:104EF0002003ECE30E94CA310895A0915403B091BD
:104F000055030895A0915203B0915303C5CEE0918B
:104F10005203F09153030895A4E6B0E00C94AD2F32
:104F2000E7EAE0937A00A4E00C949E03EF2FF0E010
:104F30006E2EE7E2E0937A000895E7EAE0937A00C4
:104F4000A3E00E949E03EF2FF0E09E2EE7E2E093A5
:104F50007A000895E7EAE0937A00A1E00E949E03B8
:104F6000EF2FF0E0BE2EE7E2E0937A000895E0E054
:104F7000F0E00E9419330895EBE0E093E503E8EBDD
:104F8000E093E6030895E8ECF0E0E0936803F09323
:104F900069030895E0EDF7E0E0936A03F0936B0393
:104FA0000895E0934203F093430308950E94A231D1
:104FB0000E9423300E94DC320895E0934803F0936E
:104FC00049030895E0936203F093630360936403DD
:104FD000709365030895E0935203F093530308958B
:104FE000AAE0B0E00C94AD2F0E949E030E9497317E
:104FF0000E9493310895E7EAE0937A00A0E00E94CE
:105000009E03EF2FF0E00895E0938803F093890367
:1050100060938A0370938B030895E0914203F091AB
:1050200043030895E0918803F091890360918A0316
:1050300070918B030895E7E2E0937A008AE48A9501
:10504000F1F708958AE48A95F1F7E7EAE0937A00A8
:105050000895A7E00E949E03EF2FF0E0E09338034D
:10506000F09339030895A0913803B091390308955E
:10507000A12FE2E30E94CF310E2E08950E2EA52D12
:10508000E1E00E94CF310E22AC8DE0E00E94AC3115
:10509000E02108950E2EA52DE1E00E94CF310E22D1
:1050A000AB8DE0E00E94AC31E0210895E4E00E9485
:1050B000CA31E0210895F0E0E0933803F09339031A
:1050C0000895E0E0E0933803E09339030895E4E0C5
:1050D0000E94AC310E2E0895AB8DE5E00E94AC31FC
:1050E0000895AA2DEAE00E94CA310E2E0895A0E08C
:1050F000F3FCA1E0E0E00E94AC310E22A22FE3E637
:105100000895E0913803F09139030895F297ADE7DF
:10511000B0E00E9418320F010895F0E0DE01919690
:10512000AE0FBF1FEC91F0E0D0010E945032E0932F
:105130003803F093390397DFA93CE0E0BE070895F8
:10514000E8ECF0E0E0933803F09339030895F0E0E1
:10515000DE019596AE0FBF1FEC91F0E084DF0E9458
:105160001832DF01E4E6F0E00E945032E0933803A9
:10517000F09339030895E02FF0E0DE015D96AE0F65
:10518000BF1F0895A0917C03B0917D0380917E03A1
:1051900090917F030895E8EEF3E060E070E00E94F4
:1051A0008D32DF01CB01ADDF662777270895EC91C3
:1051B000F0E0A0E4BCE90E945032E4DF66277727E4
:1051C0000895E0937C03F0937D0360937E037093D6
:1051D0007F030895D7DFDFCF0E947131E5E0F0E073
:1051E00060E070E00E94103208950E947131E4E1A5
:1051F000F0E060E070E00E94083208950E94713192
:10520000A431E0E0BE07E0E08E07E0E09E070895ED
:10521000E0918403F0918503609186037091870388
:10522000A0E5B4E180E090E00E944B32CACFE8EE06
:10523000F3E060E070E008950E948D32E09338035F
:10524000F09339030895A62DEAE00E94CA310E2E8C
:105250000895A22FE3E60E94CA310895A0E0F0FC71
:10526000A1E0E0E00E94AC31E0210895FCDEE0E046
:10527000F0E00E94D4310895E89425F8E0E0E0934E
:1052800022030895F0DE08CD0E22A0E022FCA1E06A
:10529000E1E00E94AC31E0210895E0932F03ECCFD0
:1052A000E0E00E94AC310E220895E0E00E94AC31B3
:1052B000E0210895E0E00E94AC310E2E0895E091C7
:1052C0000403F0E03597CFDE0E94EC310E2EE09122
:1052D0002E0303DEFF27662777270895E1E00E946B
:1052E000AC310E2E0895A0E022FCA1E0DECFEF85C8
:1052F000F889A0918803B091890380918A039091E5
:105300008B03662777270E9408320E2EEAE0F0E032
:1053100060E070E00E9410320895E0936803F0931B
:10532000690308957FDEAF85B889882799270E9491
:1053300071310895A630E0E0BE07E0E08E07E0E0BE
:105340009E070895A0916803B09169030895E091C4
:105350006803F09169030895EF85F889A0918803A7
:10536000B091890380918A0390918B0366277727F8
:105370000895E0933803F09339030895E32FA09143
:10538000CC03B091CD038091CE039091CF03FF2742
:10539000662777270E942330089565DEEAE00E94A1
:1053A00040320895E32FF0E0A091CC03B091CD03FB
:1053B0008091CE039091CF030E94A2310E942330AE
:1053C000C2CCA0916A03B0916B0308950E94A731EB
:1053D0000E94ED32B8CCA32FBB27E091CC03F09113
:1053E000CD036091CE037091CF03F0CFE0916A03BB
:1053F000F0916B0308950E94A2310E94233008951A
:10540000EAE0F0E00E946332B4CFE091160365DD7C
:10541000FF27662777270895E0937203F0937303BD
:105420000895E0911603F0E058DD0E94A2310E9439
:10543000713108950E944632A0917203B0917303B6
:105440000895E0917203F09173030895A0911603FB
:10545000BB27E0918403F0918503609186037091EE
:1054600087030E94A7310E9471310895E1E00E94F4
:10547000AC31E0210895A0E0F099A1E0E1E00E94C4
:10548000AC3134CD0E22A22FE3E60E94AC31E021F4
:1054900008950E2EA0912003ECE30E94CA310E2243
:1054A00008950E941933A1E0B0E00C94AD2FE09173
:1054B000B803F091B9036091BA037091BB03A4E300
:1054C000B0E00E94EC2FEDCFACE3B0E00E94EC2FF7
:1054D000E8CF3EDCAEE3B0E0E4CF0E942133A1E0B0
:1054E000B0E00C94AD2FEAE00E94CF310E2E08956B
:1054F000AB2DEAE00E94CA310E2EA0E027FCA1E00D
:10550000CFCEA0912B03E3E00E94AC310E2E089584
:10551000A92DEAE00E94CA310E2E0895E0910D03F4
:10552000F0E0E85FFC4F0895E0914803F0914903F3
:105530000895A22FE3E60E94AC31E0210895E091A6
:105540003503EF5FE0933503E0913403A091350319
:10555000EA1708950E94CA310E2EA0E023FCA1E0B4
:105560000895A0914803B09149030895A0915C0368
:10557000B0915D030895E1E00E94F932EA1B0E94B8
:105580004C330895A091CC03B091CD038091CE030C
:105590009091CF030895E091CC03F091CD036091F9
:1055A000CE037091CF030895A0E0B0E080E09FE3C8
:1055B0000E945D300895E093BC03F093BD036093B7
:1055C000BE037093BF030895E6DFA6E7B3E0F4CB14
:1055D000E0919C03F0919D0360919E0370919F0365
:1055E0000895EAE0F0E00E9450320895A0919C03F3
:1055F000B0919D0380919E0390919F03089587DB56
:105600008FCBE0939803F093990360939A03709380
:105610009B030895E0E00E94CF31E0210895A12F7F
:10562000B0E0EAE0F0E00E9463320895EB85FC858B
:10563000A0918803B091890380918A0390918B0394
:10564000662777270895A0918803B09189038091F8
:105650008A0390918B030895F0E0EA0FFB1FE0931B
:105660004603F0934703AEE30C9409260E940926F3
:10567000A0E00C940926E0914703AE2F0E94092672
:10568000A09146030C940926B0E0E2E0F0E00E940D
:1056900063320895DE01AF5BBF4FEC930895EAE0FB
:1056A000DE01AD5BBF4FEC930895DE01AB5BBF4FF6
:1056B000EC930895DE01AA5BBF4FEC930895DE01E1
:1056C000A95BBF4FEC930895EAE0DE01A85BBF4FF2
:1056D000EC93DE01A75BBF4FEC93DE01A65BBF4FEF
:1056E000EC93DE01A55BBF4FEC93DE01A45BBF4FE3
:1056F000EC93DE01A35BBF4FEC93DE01A25BBF4FD7
:10570000EC93DE01A15BBF4FEC930895E9E0EEA7B7
:10571000E0913103E170EE0FAE2FE0913103E69599
:10572000E170EE0FEE0FEE0FEA0F0E2E0895E091EE
:105730003103E695E695E170AE2FE0E0F5FCE1E09F
:10574000EA2BEE0FEE0FE00DEDA70895EEA7E09126
:105750003103E170EE0FAE2FE0913103E695E17079
:10576000EE0FEE0FEE0FEA0F0E2EE1CFE295E07F87
:10577000EE0FEE0F0895E0E020FCE1E0E09301037E
:10578000A0918C03B0918D0380918E0390918F0333
:105790000895A0918C03B0918D0380918E03909118
:1057A0008F030895AA30E0E0BE07E0E08E07E0E056
:1057B0009E07089592DBEAE0F0E060E070E0089573
:1057C0000E948D32DF01CB01EAE0F0E060E070E0A2
:1057D0000E94A7320895FE01E05CFF4F34960895C1
:1057E000DE01AD5BBF4FEC930895E0917403F0913F
:1057F00075030E947631DF01EAE0F0E00E94633237
:10580000E0937603F09377030895A0917603B09127
:1058100077030895FE01E05CFF4F3196BF01F5DF8D
:10582000EAE0F0E00E946332DF01EAE0F0E00E948B
:105830009532DB01EC930895FE01E05CFF4F329658
:10584000BF01E3DFEAE0F0E00E949532DB01EC9378
:105850000895A0917A03B0917B030895FE01E05C66
:10586000FF4F35960895E4E6F0E060E070E00895BB
:10587000EC93FE01E05CFF4F08958BDFEAE0F0E07F
:1058800060E070E00895A0E020FCA1E0EA2FE2953E
:10589000E07FADA5EA0FEDA70895A0914003B09178
:1058A00041030895FE01E05CFF4F3D96BF01F5CF37
:1058B000E8EEF3E00E945032DF01EAE0F0E00E94FF
:1058C0009232DB010895E4E6F0E00E945032DF01FD
:1058D000EAE0F0E00E949232DB010895FE01E05C14
:1058E000FF4F3E960895DF01EAE0F0E00E94923219
:1058F000DB0108950E949232DB01EC930895E2E00F
:10590000DE01A85BBF4FEC930895BB27EAE0F0E00F
:105910000E949532DB010895EAE0F0E00E946332D4
:10592000DF01EAE0F0E00E949532DB010895FE011C
:10593000E05CFF4F3A9608950E946832DF01CB0188
:10594000EAE0F0E060E070E00E94A3320895A03148
:10595000E7E2BE07E0E08E07E0E09E070895FE0163
:10596000E05CFF4F3B960895A83EE3E0BE07E0E011
:105970008E07E0E09E070895FE01E05CFF4F3C9635
:105980000895A436E0E0BE07E0E08E07E0E09E0761
:105990000895FE01E05CFF4F3D96089587DAEAE046
:1059A000F0E060E070E00895FE01E05CFF4F3F969C
:1059B0000895DE01A75BBF4FEC93E4E7DE01A65B31
:1059C000BF4FEC930895E0E4DE01A25BBF4FEC9380
:1059D0000895DF01CB01E0E0F0E060E171EC0E94AE
:1059E00040310895E0E4DE01A35BBF4FEC930895DE
:1059F000DF01CB01E0E0F0E066EC72EC0E944031A8
:105A00000895E0E4DE01A45BBF4FEC930895DF014D
:105A1000CB01E7C9E0E4DE01A55BBF4FEC9308953D
:105A2000A0919003B0919103809192039091930380
:105A3000089519DFC5CEF4DFEAE0F0E060E070E041
:105A40000895EEA5E058EEA7EEE3B3CFE091700322
:105A5000F09171030E947631E0937003F09371032B
:105A6000089555D9A4E6B0E080E090E096C9A091F1
:105A70007003B09171030895BF01F9DFE0E1F7E22F
:105A80000E946332DF01EAE0F0E00E949532DB0120
:105A9000EC930895BF01EBDFE8EEF3E00E94633280
:105AA000DF01EAE0F0E00E949532DB01EC9308951B
:105AB000BF01DDDFE4E6F0E00E946332DF01EAE0EF
:105AC000F0E00E949532DB01EC930895BF01CFDF37
:105AD000EAE0F0E00E949532DB01EC930895E0E506
:105AE000DE01A55BBF4FEC930895A0917803B091C0
:105AF00079030895BF01F9DFE4E6F0E00E94633224
:105B0000DF01EAE0F0E00E949532DB01EC930895BA
:105B10003F96BF01EADFEAE0F0E00E949532DB0148
:105B2000EC930895DE01A75BBF4FEC930895DE016F
:105B3000A65BBF4FEC930895DE01A55BBF4FEC93CE
:105B400008950E946332DF01EAE0F0E00E9495329E
:105B5000DB01EC930895EAE0F0E00E9495320895AD
:105B6000ED85FE85F695E79508950E945032BBCEEF
:105B7000A0914C03B0914D030895EAE0F0E0BACE55
:105B8000DE01A35BBF4FEC930895DE01A25BBF4F24
:105B9000EC930895DE01A15BBF4FEC930895E9E318
:105BA000C6DFE8E3C9CFE170EE0FEE0FEE0F089508
:105BB000ECE7BDDF94CFECE0DE01A45BBF4FEC93DC
:105BC0000895DE01A45BBF4FEC930895AB8DE4E034
:105BD0000E94AC31AE2FE0E020FCE1E0EA23089522
:105BE000AE2FE0E020FCE1E0EA230895ECE7C8DF17
:105BF000E0E5CBCFE7E7C4DFE9E3C7CFE52FF0E08F
:105C0000DE01A05CBF4FAE0FBF1F08950E94AC31F4
:105C10000E2EAE8108950E94AC310E2AAE810895F9
:105C2000AE81E2E30E94AC310E2EA989BA89E4EA82
:105C3000F1E00895BF01A989BA89D3CCAE81E5E02E
:105C4000E5CFE3E10E94AC31E0290895E72DF0E0D3
:105C5000DE015D96AE0FBF1F0895A0918003B09145
:105C6000810380918203909183030895EC91F0E089
:105C7000A0E4BCE90E945032F0DF66277727089540
:105C8000E0938003F0938103609382037093830316
:105C90000895E3DF80CAE0918403F0918503609169
:105CA000860370918703A0E5B4E180E090E00E9454
:105CB0004B32E6CFC8DCEAE0F0E060E070E0089547
:105CC00020DAF695E79555CBECA7CDD9A436E0E0E0
:105CD000BE070895BF01C7D9F6CDFE01E05CFF4FB6
:105CE0003696BF01C0D97DCCFE01E05CFF4F3796F0
:105CF000BF01B9D942CFBF01A0915A03B0915B0354
:105D00000895E9E30FDFE0E512DFEEE315CFBF0111
:105D1000A0914403B09145030895A0915003B09120
:105D200051030895FE01E05CFF4F37960895A0915E
:105D30003A03B0913B030895E170E795E0E0E79501
:105D4000AE2F0895FE01EB5BFF4FE0810895E295D1
:105D5000EF70E695E1700ADDEA2BAE2F0895E2952B
:105D6000EF70E695E695E170E295E07FEE0FEA2BA5
:105D7000AE2F0895E295E170E295E07FEA2BAE2F19
:105D80000895EA2BAE2FDECFE695E170EE0FEE0F11
:105D90000895E695E695E170EE0F0895E695E6958F
:105DA000E695E170EA2B0895FE01EA5BFF4FE08182
:105DB0000895FE01E95BFF4FE0810895EA2BAE2FC5
:105DC000F8CFEA2BAE2FF0CFFE01E75BFF4FE0816B
:105DD0000895FE01E35BFF4FE0810895E695E170D1
:105DE000C5DCEA2BAE2F0895E695E695E170E295C5
:105DF000E07FEE0FEA2BAE2F0895E695E695E69547
:105E0000E170E295E07FEA2BAE2FEEA50895E695CE
:105E1000E695E695C8CEEA2BAE2FDBCFE295EF7084
:105E2000E695E170EE0FEE0F0895E295EF70E695BE
:105E3000E695E170EE0F0895FE01E45BFF4FE0810F
:105E40000895EA2BAE2FFE01E25BFF4FE08108953B
:105E5000E295EF70E69570CFFE01E55BFF4FE081C4
:105E60000895EA2BAE2FF8CFFE01E25BFF4FE081F1
:105E70000895E295EF70E695E6950895FE01E65BDC
:105E8000FF4FE0810895EA2BAE2FFE01E15BFF4F4B
:105E9000E0810895EA2BAE2F97CFFE01E15BFF4F23
:105EA000E0810895E170E295E07FEA2B0895AE2F3E
:105EB000FE01EF5BFF4FE0810895E170EE0FEE0F02
:105EC000EA2B0895E17052DCEA2B0895E695E17023
:105ED000E295E07FEE0FEA2B0895E695E695EDCF8B
:105EE000E170EE0FEA2BAE2F0895FE01EE5BFF4F3F
:105EF000E0810895E295EF70E695D4CFFE01ED5B69
:105F0000FF4FE0810895AE2FFE01EC5BFF4FE08173
:105F10000895FE01EC5BFF4FE0810895289885E22B
:105F20008A95F1F751E008955E9885E28A95F1F738
:105F3000ECE0E51B089585E28A95F1F75E9A85E22B
:105F40008A95F1F708955D9A85E28A95F1F7289A86
:105F500084E191E00197F1F7E1CF109639F08DECF3
:105F60009AE00197F1F7A8951197C9F7089530972E
:105F70006040704009F070580895552342F450383D
:105F800011F4E0FF04C03196691F791F6BF050E8EF
:105F9000572711F45F93CFC05F3F31F0660F000CBD
:105FA00057956795752F08955F9300200AF0CFC02D
:105FB000C8C050E8192E1522880F991F9527550F34
:105FC000879550E8072E0522660F771F7527550F16
:105FD00067950895689401C0E8945F93F2DF703884
:105FE00018F07F3F08F4A7C056E1571BAAF451955B
:105FF00058300EF4593030F0EFEFFFEF6FEF7FE7DE
:1060000077F91AC077275523B9F0EE0FFF1F661FE7
:10601000771F5A95D1F710C07727583028F0EF2F07
:10602000F62F672F5850F9CF552331F076956795A5
:10603000F795E7955A95D1F700200AF45BD15F9167
:106040000895689401C0E894309760407040B1F0C2
:10605000002426F0772312F400944CD1172E7EE111
:10606000112032F07A95EE0FFF1F661F111CF9CF39
:10607000EF2FF62F612D5F938ADF5F9108954F9385
:10608000AF01FD01DA01AB01BC01CA01402D012CB9
:10609000142E4F910895EA0FFB1F681F0895E09595
:1060A000F0956095EF5FFF4F6F4F08955F9381DF2D
:1060B000903871F150E8152604C05F937ADF90386C
:1060C00039F1703821F1572F591B2BF112F4D7DF1A
:1060D000FACF583118F0AA27BB278827583028F064
:1060E000AB2FB82F88275850F9CF552329F0869524
:1060F000B795A7955A95D9F7502D512572F0CBDF5A
:1061000038F46795F795E795739513F420C0B7DFDA
:106110003EDF5F910895D8F7FBCFEA1BFB0B680BBE
:1061200051F010F40094BBDF662392F3EE0FFF1FD3
:10613000661F7A95CBF7EE27FF27662777275F91B3
:106140000895EFEFFFEF6FE77FEF5F910895EFEFB7
:10615000FFEF6FE77FE75F9108955F932ADF703865
:1061600051F3903841F301240894791F23F41CF370
:1061700000203AF3ECCF0F921F932F933F934F934E
:10618000112722279927689FA0018F9F302D410D4D
:10619000591F6B9F300D411D591F8E9F27D0BF9FE8
:1061A00025D06A9F23D0BE9F1DD0AF9F1BD0AE9F2E
:1061B000110D291F391F491F591FE32FF42F652F78
:1061C000522F4F913F912F911F910F9066232AF0EC
:1061D000550FEE1FFF1F661F02C073954BF2CDDEF9
:1061E0005F910895100D211D391F02C0200D311D32
:1061F000491F591F08955F93DCDE703821F4112088
:106200000AF49FCFA4CF903809F495CF01240894C5
:10621000970B1BF4D4F30020F3CF792F1F932F9308
:106220003F934F93112411272227332744275527C3
:1062300090E2AE17BF078607410730F0AE1BBF0BD9
:10624000860B410B089401C08894551F221F331FF1
:10625000111CAA1FBB1F881F441F9A9551F7F901F3
:10626000612D4F913F912F911F91662332F0550F71
:10627000EE1FFF1F661F7A9543F27FDE5F91089540
:1062800099239AF0772342F0971748F029F4AE1734
:10629000BF07860720F031F0989488940895989469
:1062A000089408951894889408957723C2F797174F
:1062B00098F3A9F7EA17FB07680788F399F3ECCF7F
:1062C000DFDFE1E009F008F0EE270895D9DFE1E033
:1062D00009F008F4EE270895EA0FFB1F681F791FE5
:1062E0000895AE1BBF0B860B970B0895F195E195B2
:1062F000F0400895F09560957095E195FF4F6F4FD0
:106300007F4F0895EE230E2EEA2F19F0E6950A949A
:10631000E9F70895EE230E2EFD0121F0F695E7959D
:106320000A94E1F70895F695E795F695E795F695C1
:10633000E795F695E7950895FE2FFF0FFF0B6F2F5A
:106340007F2F08956F2F660F660B762F08958B2F82
:10635000880F880B982F0895EA17E1E009F0EE27DF
:106360000895EA17E1E009F4EE270895AE17E1E099
:106370000CF4EE270895AE17E1E00CF0EE27089537
:10638000EA17E1E00CF0EE270895AE17E1E008F41B
:10639000EE270895AE17E1E008F0EE270895EA171A
:1063A000E1E008F0EE270895EA17FB07E1E009F0C5
:1063B000EE270895EA17FB07E1E009F4EE270895B8
:1063C000AE17BF07E1E00CF0EE270895EA17FB07D0
:1063D000E1E00CF0EE270895AE17BF07E1E008F00A
:1063E000EE270895EA17FB07E1E008F0EE2708958D
:1063F000EA17FB0768077907E1E009F0EE2708953F
:10640000EA17FB0768077907E1E00CF4EE27089527
:10641000AE17BF0786079707E1E00CF0EE27089557
:10642000EA17FB0768077907E1E00CF0EE2708950B
:10643000FA9FF02DEB9FF00DEA9FE02DF10D0895EE
:106440007A9F702D6B9F700DF89F700DE99F700DF6
:106450006A9F602D710DFB9F600D711DE89F600D9F
:10646000711D8827FA9FF02D610D781FEB9FF00DAD
:10647000611D781FEA9FE02DF10D681F781F0895B8
:106480006E2F6A9FF0016B9FF00D089574D0D0DFDE
:106490000EF42CDF08957DD0D3DF0EF42BDF0895AA
:1064A0000024112490E1AA0FBB1F001C111C0E1A1E
:1064B0001F0A18F40E0E1F1E01C0A1609A9599F7CD
:1064C000FD01D001089557D0EBDF0EF40FDF0895E2
:1064D0003F934F935F93002411244427552730E2C4
:1064E000AA0FBB1F881F991F001C111C441F551F9A
:1064F0000E1A1F0A460B570B28F40E0E1F1E461FBE
:10650000571F01C0A1603A9559F7FD01BC01D001A8
:10651000CA015F914F913F9108953BD0D9DF0EF4AE
:10652000E9DE0895BDDFFD010895E894B7FF04C0DA
:10653000A095B09511966894F7FDD8DEB1DFFD0106
:106540000EF4D4DE0895C4DFFD01BC010895E89483
:1065500097FF09C0A095B09580959095AF5FBF4F0C
:106560008F4F9F4F689477FDC5DEB2DFFD01BC0100
:106570000EF4C0DE0895E894F7FF02C0B7DE689419
:10658000B7FF06C0A095B095119600F8039400FAE5
:106590000895E89477FF02C0ADDE689497FF0BC0C2
:1065A0000024A095B095809590951196801D901D22
:1065B00000F8039400FA0895ED93FD936D937C9396
:1065C0000895A881B9818A819B810895E883F98320
:1065D0006A837B830895689401C0E89401D034DD18
:1065E000182E862F612D192E972F712D1B2EBF2F40
:1065F000F12D1A2EAE2FE12D0895129602D0BF0173
:106600001297119602D0FE2F1197F999FECFFF93A2
:10661000FFB7F894A1BDB2BDF89AE0B5FFBFFF91F6
:10662000089507D012960F01FB0103D0F0011297D5
:10663000089507D01196EF93EF2F03D0EF911197A4
:106640000895F99B02C0A895FCCF9FB7F894A1BD0F
:10665000B2BDF89A80B5E81719F0E0BDFA9AF99A38
:106660009FBF089500240E160F060606070608951C
:1066700000240A160B06089500240A160B060806C5
:1066800009060895EA17FB07680779070895AE170A
:10669000BF07860797070895E894EE2309F06894EA
:1066A0000895AC0FBD1F05900D928A95E1F70895EE
:00000001FF
